:100200004F726967696E616C2046696C653A20704F
:10021000726F6A6563742E6865780D0A4F75747025
:10022000757420446174653A20323030392F303390
:100230002F30390D0A4F75747075742046696C65DE
:100240003A206B6C39372E6865780000000000009A
:10025000000000000000000000000000000000009E
:10026000000000000000000000000000000000008E
:10027000000000000000000000000000000000512D
:107FF6000D0A0D0A205B4B4C39375D0D0A0D0A0040
:108006000D0A0D0A00557365204B4C39374320493C
:108016004F20446566696E650D0A005365742041FC
:1080260064383139782053776974636820526567FC
:1080360069737465720D0A005365742041643831A2
:108046003978205377697463682052656769737459
:10805600657220446F6E650D0A0052656D6F74651A
:1080660020696E2052554E206D6F64650D0A0052D0
:10807600656D6F7465205061737320434841206BB2
:1080860065790D0A0052656D6F74652050617373D2
:1080960020434842206B65790D0A0052656D6F7466
:1080A60065205061737320434843206B65790D0A40
:1080B6000052656D6F7465205061737320434844A8
:1080C600206B65790D0A0002800040001000200038
:1080D60001000200040000028000400010002000A1
:0780E6000100020004000884
:1087CC0041FA780041F9040041F90B0041F903002A
:0C87DC0041F9010041F9020041FA8B0054
:1085590074FF90F90CF07B017AF9790C90FD97E49E
:10856900F0A304F0227401F0A374F9F0742EA3F0BF
:10857900A37401F0A32290FDAFE0FF7401A80708DE
:10858900227B0190FD97F0A304F0E4FD7F942290F3
:10859900FDAEE075F021A42412F582E5F034F9F579
:1085A90083E02290F904E090F90BF022EF75F021B5
:1085B900A4240DF974F935F0FA7B01227401F0A3B2
:1085C90074F9F0A3744F2290F903E090F901F022B5
:1085D90090FDAEE0FFC32290FDAEE004F022A4249A
:1085E9000DF582E5F034F9F583E0227B017AF9791A
:1085F90001227401F0A374F9F0A3740DF022A3F021
:108609007B017AF9790722A3F07B017AF9790922AA
:108619007B017AF979052290F903E0FF90F901E0ED
:01862900222E
:1034EB00E490FDAEF0A3F0A374FFF0A3F0E4A3F01F
:1034FB00A3F07F0512B33DE4F5207DFF7F05127924
:10350B007C7B027DFF7F051267107D1E7F02127987
:10351B007C7B027D1E7F021267107D037F06127873
:10352B00157B027D03123AEE7D017F0A126710E4D0
:10353B00FB7D037F0C126710E4FB7D0F7F0112678D
:10354B0010E4F5F1FB7D04123AEE7D087F0612675D
:10355B0010D2AF75FF387BFF7AB2791E12B349E4F4
:10356B00FF12A9397D017F407E0212915F7BFF7AAA
:10357B007F79F612A4937BFF7A02790012A4937BD6
:10358B00FF7A80790612A4937BFF7AB379AF7F031E
:10359B0012B36B7B007C077DD01276AA7BFF7A80FF
:1035AB00790B12A49390FE0574FFF0A37480F0A323
:1035BB0074DDF07B017AF8790012AB517D0C7F0B37
:1035CB0012797C7B017D0C7F0B1267107D017F08CC
:1035DB0012797C7B027D017F081267101295127D98
:1035EB00017F081278157F0112B33D7B017AF979BF
:1035FB000DE4FD1280ED7AF9792E7DB4123AC67A7C
:10360B00F9794F7DB91280ED7AF979707DE0123A34
:10361B00C67AF979917DE51280ED7AF979B27DEA76
:10362B00123ADE7AF979D37DEF1280ED7AF979F4DB
:10363B007DD0123ADE7AFA79157DD51280ED7B01B9
:10364B007AFA79367DDA1280ED7B017AFA79577D39
:10365B00DF1280ED7FE012B3A31286197D701292F8
:10366B00A01286097D7E1292A01286127D7C129288
:10367B00A07AFA79797D60123ACE7AFA797B7DE07D
:10368B00129D8F7AFA797D7DE2123ACE7AFA797FA2
:10369B007DE4129D8F7AFA79817DE6123AF67AFAF9
:1036AB0079837DE8129D8F7AFA79857DEA123AF655
:1036BB007AFA79877DEC129D8F7B017AFA79897D75
:1036CB00EE129D8F90FCFD1285FBA312856E128569
:1036DB00C9F01286191293DC90FCFD12856E74F9F9
:1036EB00F0747012857774F9F07491128607129347
:1036FB00DC90FD0912856E74F9F0A374B212857813
:10370B0074F9F074D31286071297E990FCFD1285B9
:10371B00C512857874F9F0A374F412857874FAF0F5
:10372B0074151286101293DC90FD091285C5128553
:10373B007874FAF0A3743612857874FAF074571211
:10374B0086101297E990FE0B1285FB7B017AFA79B2
:10375B007912B26DE490FDAEF01285D99408503F0A
:10376B00EF75F002A4247BF974FA35F0FA7B01C0F3
:10377B0003C002C0017E007C007D211217E0747033
:10378B002FF974F93EFA90FE0BEBF0A3EAF0A3E9E4
:10379B00F0D001D002D00312B26D1285E080BAE4F2
:1037AB00FFFE12B1C7EFD39403E4400690FE3AF04C
:1037BB00800AFFFE12B1C790FE3AEFF090FE3A740A
:1037CB0001F07BFF7A80792112A493744012855B00
:1037DB00E4FD7F9412896612855FFD7F94128966E2
:1037EB0090F90C7401F0FB1285617D107F941289A6
:1037FB00661285597D117F9412896612855F7D1241
:10380B007F941289661285597D137F9412896612F3
:10381B00855F7D147F9412896690F90C7403128571
:10382B005E7D207F941289667BFF7A80793E12A49D
:10383B0093200803023AC0C20890FDAE7403F0E473
:10384B00A3F01285D9940B40030238FA75F021EFDF
:10385B001285E7FB7039128598FC30E40C12857FDA
:10386B008002C333D8FC0238D9EC30E51790FA78D4
:10387B00E075F01484E5F0706C12857F8002C33321
:10388B00D8FC803912857F8002C333D8FC8050EB83
:10389B006405600E90FDAEE075F0211285E7640CB7
:1038AB00703412859830E61D90FA78E075F0288414
:1038BB00E5F0703112857F8002C333D8FCFD7F05A4
:1038CB001269EC802012857F8002C333D8FCFD7F08
:1038DB000512797C800F12857F8002C333D8FCFDE3
:1038EB007F051278151285E0A3E004F002384D90A5
:1038FB00FA78E004F0C394C84002E4F07B017AF953
:10390B00790D123AFE90FDAE7401F01285D9940335
:10391B00500B1285B51255471285E080EE90FDAE27
:10392B007403F01285D9940B500B1285B5122186B6
:10393B001285E080EEE520F460657D0F7F01129427
:10394B007990F904EFF0700A12AAECE490F901F007
:10395B0080491285AC5408FFF0BF080790F9037437
:10396B004380311285AC5404FFF0BF040790F90378
:10397B00744280201285AC5402FFF0BF020790F90D
:10398B00037441800F1285AC5401FFF0BF010B9003
:10399B00F9037440F012A6D38005E490F903F0E527
:1039AB0020B4FF0D7D027F06127815123AD6023A2B
:1039BB00377D027F0612797C12861912AB1FEF60DE
:1039CB004390F901E0FCB44307123AD67D028027FD
:1039DB00ECB44207123AE67D04801C90F901E0FC3E
:1039EB00B44107123AE67D08800DECB4400E7D1E03
:1039FB007F021278157D107F0212797C90FDB274D4
:103A0B0001F080287D1E7F0212781590FDB3E0D364
:103A1B0094C85005E004F0801390FDB2E0B40103AC
:103A2B0012A7D0E490FDB3F090FDB2F090FDB0E0A2
:103A3B0025E0F0E0FE7D047F06129479EF60047FB1
:103A4B000180027F00EE4FFF90FDB0F0BF7F0EE5CF
:103A5B0020B4FF047F1D80027F0212006E90FDB127
:103A6B00E025E0F0E0FE7D087F06129479EF60041C
:103A7B007F0180027F00EE4FFF90FDB1F0BF7F050D
:103A8B007F0412006E30090AC2097F0112AE4F1279
:103A9B00006E1240A4200D0302383C90FA8BE0FF1D
:103AAB0004F0EFD39464500302383CC20D7F1D1217
:103ABB00006E02383C43870102383C7B011280EDDB
:103ACB007B01227B01129D8F7B01227D1E7F0212C7
:103ADB007815227B011280ED7B01227D1E7F021265
:103AEB007815227F06126710E4FB227B01129D8F53
:033AFB007B01222A
:10006E00E490FEF0F0EF1470030201B71460261452
:10007E0070030201D214700302012324F2601824CB
:10008E00F870030201AC24FE70030201C214600377
:10009E000201E480438004E520703D7520FF7B0162
:1000AE007AF9797012B3557AF9799112B3557AF9C2
:1000BE0079B212B3557AF979D312B3557AF979F434
:1000CE0012B3557AFA791512B3557AFA793612B304
:1000DE00557AFA795702B355E4F5207B017AF9790E
:1000EE007012B3607AF9799112B3607AF979B2121B
:1000FE00B3607AF979D312B3607AF979F412B360F6
:10010E007AFA791512B3607AFA793612B3607AFAFE
:10011E00795702B3607BFF7A80796012A49390F9CD
:10012E0001E090F903F090F9027401F090F903E008
:10013E0064406005E014F0800690F9037443F0907B
:10014E00F903E0FFB4400890FEF07401F08022EF56
:10015E00B4410890FEF07402F08016EFB44208909D
:10016E00FEF07404F0800AEFB4430690FEF07408BB
:10017E00F07D0F7F0112947990F904EFF090FEF06C
:10018E00E05FF0600C1285D012A52D90F902740478
:10019E00F090F902E004F0E0D39404408F227A80CC
:1001AE0079751201E5744380297A80798B1201E505
:1001BE007442801E7BFF7A8079A112A49390F9037A
:1001CE007441800E7BFF7A8079B712A49390F90365
:1001DE007440F012A713227BFF12A49390F903220E
:10A6D300128620FD6F6038EDB443047E08801AEDC6
:10A6E300B442047E048012EDB441047E02800AED7C
:10A6F300B440047E018002E4FE7D0F7F0112947951
:10A7030090F904EFF05EFE70061285D012A52D229B
:10A713001286206F6038EFB440047E01801AEFB4D4
:10A7230041047E028012EFB442047E04800AEFB437
:10A7330043047E088002E4FE7D0F7F01129479902A
:0FA74300F904EFF05EFE60061285D012A52D22FC
:10A52D00E490FEF1F0F07AFE79F112858A128966D7
:10A53D007B017AFE79F112856512A5717F0112B347
:10A54D003D1285F4128565E412A5711285F412850C
:10A55D0065FD7F941289667F0212006EE490FA8B7E
:0BA56D00F0D20D22FD7F9412896622BF
:10A7D000E490FEF2F0F07AFE79F212858A12896630
:10A7E0007B017AFE79F2128565FD7F941289667F7E
:10A7F0000112B33D1285F4128565E4FD7F94128940
:0DA80000661285F4128565FD7F940289665D
:10AAEC00E490FEF3F0F07B017AFE79F312858C1280
:10AAFC0089667B017AFE79F3128565FD7F94128954
:10AB0C00667F0112B33D7F0212006EE490FA8BF067
:03AB1C00D20D2235
:10B21E00AE07E4FF12AE4FBF0109EE7006EDB4109B
:04B22E0002D209221D
:03B3AF00D208229F
:104B32000000000000000000000000000000000073
:104B42000000D60980A020E02D101060A20004030E
:104B5200000000188C0AD08A20E02D10103E96002A
:104B62000403000000188C0AD08A20E02D10103EA9
:104B72009600100900000018011D007251D01E207D
:104B82006E28550010090000001E011D8018711CBE
:104B92001620582C250010090000009E8C0AA01433
:104BA20051F01600267C43000403000000988C0A92
:104BB200A01451F01600267C430010090000009852
:104BC2008C0AA01451F01600267C43000403000056
:104BD20000188C0AA01451F01600267C430010091C
:104BE2000000001818154028B2F016004CF84300D7
:104BF20004030000009818154028B2F016004CF883
:104C0200430010090000009818154028B2F0160061
:104C12004CF8430004030000001818154028B2F0B5
:104C220016004CF843001009000000181815A014D3
:104C320051E02D10207C9600040300000018181586
:104C4200A01451E02D10207C9600100900000018DD
:104C5200023A801871382D40582C45001009000086
:104C6200001E8C0AD090204031200C4055000403D5
:104C7200000000188C0AD090204031200C405500D2
:104C8200100900000018011D00BC52D01E20B828D7
:104C9200554010090000001E011D80D0721C162014
:104CA200102C258010090000009E8C0AA0205120A3
:104CB2001810187E23000403000000988C0AA0201C
:104CC20051201810187E23001009000000988C0A49
:104CD200A02051201810187E2300040300000018A1
:104CE2008C0AA02051201810187E23001009000001
:104CF200001818154040B220181030FC230004039D
:104D02000000009818154040B220181030FC230013
:104D120010090000009818154040B220181030FC0D
:104D2200230004030000001818154040B220181098
:104D320030FC23001009000000181815A020514073
:104D420031201880550004030000001E1815A02011
:104D5200514031201880550010090000001E023A0F
:104D620080D072382D40102C458010090000001EA2
:104D7200011D803E73382D407E2C458010090000B5
:104D8200001E011D80D072382D40102C4580100964
:104D92000000001E011D80D072382D40102C45806D
:104DA20010090000001E3B2A4028B2E02D1060F8D6
:104DB20096000403000000183B2A4028B2E02D10A0
:104DC20060F89600100900000018302A4040B240F6
:104DD200312030005510040300000018302A4040F2
:104DE200B240312030005510100900000018201C7C
:104DF2008080711C552020A8750410090000009ABB
:104E0200023A80D0721C1620102C25801009000056
:104E1200009E023A00BC52D01E20B828554010090C
:104E22000000001E1815D090204031200C40550083
:104E32000403000000181815D090204031200C40C7
:104E420055001009000000181815D09020201810E5
:104E5200187E23000403000000981815D09020202B
:104E62001810187E2300100900000098023A8018DA
:104E7200711C1620582C250010090000009E023AD1
:104E8200007251D01E206E28550010090000001E2D
:104E92001D15D08A20E02D10103E9600040300005C
:104EA20000181D15D08A20E02D10103E9600100922
:104EB200000000181D15A01451F01600267C4300B6
:104EC2000403000000981D15A01451F01600267C62
:104ED2004300100900000098302AD0902040312071
:104EE2000C405500040300000018302AD0902040E6
:104EF20031200C405500100900000018302AA02073
:104F020051201810187E2300040300000098302A54
:104F1200A02051201810187E2300100900000098CC
:104F22003B2AD08A20E02D10103E96000403000098
:104F320000183B2AD08A20E02D10103E960010095E
:104F4200000000183B2AA01451F01600267C4300F2
:104F52000403000000983B2AA01451F01600267C9E
:104F6200430010090000009800FFFFFFFFFFFF0051
:104F72001710010901000000000E0103807341783F
:104F82002A7C119E59479B271050540000000101B2
:104F92000101010101010101010101010101011DE3
:104FA200007251D01E206E28550010090000001E0C
:104FB2008C0AD08A20E02D10103E960004030000D7
:104FC2000018000000FC0045502D48444D492D5268
:104FD200580A2020000000FD003B3D0F2E08000A69
:104FE20020202020202001D402031D714A840513B1
:104FF200140102031112102309070783010000653F
:10500200030C001000023A801871382D40582C45CC
:105012000010090000001E011D8018711C16205886
:105022002C250010090000009E011D00BC52D01E5C
:1050320020B828554010090000001E011D80D072C2
:105042001C1620102C258010090000009E8C0AD00E
:1050520090204031200C405500040300000018004D
:08506200000000000000001E28
:0687E80041FE3A00C12F22
:10506A0090FC76E0FBA3E0FAA3E02480F9E43AFAA4
:10507A00EEFF7E0029F9EE3AFA121766FD90FC8DD2
:10508A00E0FBA3E0FAA3E0F990FC88E0F5827583DF
:10509A0000ED1217BEEF2481FFEE33FE90FC76E09E
:1050AA00FBA3E0FAA3E0F98F828E8312177FFF90A9
:1050BA00FC88E02401FDE433FC90FC8DE0FBA3E0D6
:1050CA00FAA3E0F98D828C83EF1217BE90FC7FE081
:1050DA0090FC762482FFE433FEE0FBA3E0FAA3E02F
:1050EA00222480F9E43AFA90FC7FE0FF7C0029F957
:1050FA00EC3AFA121766541FFEEF2E90FC81F090DC
:10510A00FC7EE004F0A3E004F090FC76A3E0FAA3AE
:10511A00E02480F9E43AFA90FC7FE022E92480F95D
:10512A00E43AFAEE7E0029F9EE3AFA021766FF909F
:10513A00FE3CE02FFF90FE3BE03400FEE92FF9EA47
:10514A003EFA121766FF90FC7EE02480FDE433FCF1
:10515A0090FE3CE02DFD90FE3BE03CFC90FC792269
:10516A0090FC87E0FF90FE3BE0FCA3E0FDC39F7448
:10517A0080F8EC64809822F98D828C8302177FF97B
:10518A0090008212177FC3FF90FC7FE0FE9F22F9F6
:10519A008F828E8312177F90FC7E541F04FFE02FAC
:1051AA00F02290FC7EE02480FFE433FE90FC79221A
:1051BA002480F9E43AFAE92FF9EA3EFA121766FF6F
:1051CA0090FE39E02FF090FE3CE004F022FE04F05D
:1051DA00EE7C0029F9EC3AFAEF0217ACF98F828ECD
:1051EA008302177FF990008212177FFF90FC7EE0FE
:1051FA00FE2290FC7FE0FE90FC81EF541FFFEE2F11
:10520A00F022E41217BEE490FE39F090FE3BF0A3C0
:10521A00F022EE2480F582E433F58312177FFF54DF
:10522A00E022F97E007F8012174090FC7D7401F025
:10523A002290FE3BE0FEA3E0FF22541F04FF90FCF5
:10524A007FE02FF022F990008312177F54C04401A7
:10525A0090FC86F090FDB77401F0A374FCF0A3747F
:10526A0087F090FC8A22F9900001E41217BE9000A0
:10527A0002E41217BE90FDC37401F0A374FCF0A3FC
:10528A007489F090FC932290FE3BE004F02204F033
:10529A00EE2480FDE433FC90FC7922FF7C0029F99E
:1052AA00EC3AFA021766EF75F012A42432F9744B3D
:1052BA0035F0FA7BFF22FF90FC88E02402FDE433FC
:1052CA00FC90FC8D22E429F9EA3401FA121766549B
:1052DA00FE1217AC90FC7622FF90FE3CE02FFF9066
:1052EA00FE3BE03400FEE92FF9EA3EFA121766FFA8
:1052FA00222448F9E43AA801FCAD0322F98D828CF4
:10530A0083EF0217BE900001740C1217BE900002C0
:10531A00E41217BE74109000031217BE9000042204
:10532A00EF541FFFEE2F90FC80F02290FC89F9E0E9
:10533A00FE04F08E82758300EF0217BEFF04F07E32
:10534A0000E92F227E007F1212174090FC85E0228E
:10535A00F990007E02177F90FC7F7404F02290FC83
:10536A007FE0FF7E0090FE3BE0FCA3E0FD2FFFEE16
:10537A003CFE90FC81E0FBD3EF9B7480F86E982290
:10538A00E0FFC390FE3CE09F7480F890FE3BE0642F
:10539A00809822E429F9EA3401FA021766F9EF90B3
:1053AA0000010217BE90FC81E0FF90FC7FE02254CE
:1053BA001FFEEF2E90FC81F090FC7EE004F0225458
:1053CA007FFFEE2480FDEC33FC90FC7922900001F3
:1053DA00F912177FFF90FC7622541FFF90FE3CE0E3
:1053EA002FF090FE3BE034002290FC7EE0FF7E002E
:1053FA00ED2FFFEE3CFE90FC80E0FDD3EF9D748024
:10540A006E982290FC7EE02480FFE433FE90FE3CFE
:10541A00E02FFF90FE3BE03EFE90FC792290FC7F5D
:10542A00E004F022F9EF9000020217BE90FC7E74AD
:10543A0004F02274802DF582E43CF58302177FEB99
:10544A00F0A3EAF0A3E9F022C3947FEE648094808B
:10545A0022FF90FC7EE02482222FF582E43EF5832F
:10546A0002177FE0FF7E00EE90FE3BF0A3EFF022F2
:10547A0090FE39E014F4FF22F990008202177FF9B6
:10548A0090010002177FF912177F4FFF90FC9622B6
:10549A00F98F828E83E40217BE90FC88E02403F021
:1054AA0022F990007E74010217BE90FC82E0C39438
:1054BA000222F990FC88E0F582758300ED0217BE9E
:1054CA00F912177FFF90FC792290FC7EE0FF7E00A4
:1054DA002480FDEE33FC22A3F0A3EBF0A322248068
:1054EA00F9E43AFA22F974011217AC90FC9022906E
:1054FA00FC7FE02403F02290FC80E0FF90FC7EE039
:10550A00D39F2290FC7EE02403F022EF2481FFEE59
:10551A0033FE90FC7922C390FC89E0940522900026
:10552A00011217BE90000222F8AC02AD03A32212A8
:0D553A0017AC90FC932290FE3AE06403222F
:109A0C0090FE7112544990FE711250E3F8AC02AD05
:109A1C00037BFF7A4F796A7E017F00121740125246
:109A2C001012523B125452501390FE711250E3120A
:109A3C0051E61251C970EA12529180E512547A9093
:109A4C00FE711250E3F990007FEF12520D12523B4F
:109A5C00125452501090FE711250E31251BA70ED24
:109A6C0012529180E812547A90FE711250E3F990E0
:109A7C0000FFEF1217BE12539D44011217AC4402A3
:069A8C001217ACC22F22EC
:1096D10090FE7412544990FE741250E312535A646E
:1096E10001707690FE3BF0A37404F090FE7412506A
:1096F100E312548212516E504F12543D54E0646093
:10970100701F748112543F6403703212523B2482E1
:10971100125464640C70267483125463701F7F01A9
:109721002290FE741250E3F990FE3CE02480FF1277
:1097310053EC8F82F58312177F1253E3F01251D04D
:1097410070A91252910296EC90FE741250E31254D9
:0C9751008212538B40037F00227F002215
:109FB90090FE7712544990FE771250E312535AC318
:109FC9009401404E90FE3BE4F0A37404F090FE77B8
:109FD9001250E312548212516E502112543DFB5417
:109FE900E0FFBF6008ED2480FFE43CFE22EB125342
:109FF900E3F01251D070D612529180D190FE7712AF
:10A0090050E3125482FFC3ED9F7480F86C984002AC
:06A019008000E4FEFF22BE
:10AB820074811217AC74021253A9740312543074F4
:10AB92001112532074121217BE900005740412177A
:0DABA200BE90FDB71250E3F974060217AC27
:10B0EC0074091217AC740712552874071217BE9006
:0BB0FC00FDBD1250E3F974030217AC15
:10B1210074031217AC12530FE41217BE90FDC31231
:08B1310050E3F974050217ACAC
:1002800090FC76125449E490FC7DF07B0190FC8A4E
:1002900004F0A374FFF074801254E174FFF074BC96
:1002A0001254E174FFF0A374E9F0A3EBF0A374FF20
:1002B000F0A374ECF0A3EBF0A374FFF0A374F8F0D8
:1002C00090FE3AE0640260030203C590FC7612508F
:1002D000E312548920E0030215AF1252CF1250E30B
:1002E0001255321250E312522C90FC791250E31244
:1002F000535A640160030215AF90FC761250E3126A
:10030000548920E1030215AF12539D54FD1217AC1E
:1003100090FC791250E31254E8C003C002C001906F
:10032000FC761250E324801252FDD001D002D0039B
:1003300012522DE490FC7CF060030215AF12536161
:1003400090FC761250E312518940030215AF12510E
:1003500026FF54E064607058EF541FC394075003A5
:100360000215AF125427E0FF2485FDEE33FC90FC0C
:1003700076A3E0FAA3E02DF9EA3CFA121766548F4F
:100380001255391250E3F990000612177FFDC394FD
:100390001E500280027D1EEF2486FFE43EFE90FC8C
:1003A000761250E3F98F828E83ED1217BE0215AFDD
:1003B00090FC761250E312511B12512E90FC7F12CA
:1003C00051A402034090FC791250E312535AD39483
:1003D0000140037F002290FC761250E312548930D2
:1003E000E00F1252CF1250E31255321250E3125264
:1003F0002C90FC761250E39000231254CA1250E362
:100400009000231254901250E3F9EF1252DB125075
:10041000E39000241254CA1250E390002412549026
:100420001250E31253A790FC761250E3F990002586
:100430001254CB1250E3F99000251254911250E35C
:1004400012542EE412521512523BC3943CEE6480B7
:100450009480501390FC8A1250E312549A1251D097
:1004600070E512529180E0E412521512523BC3948F
:100470002DEE64809480501390FC8D1250E3125442
:100480009A1251D070E512529180E0E41252151286
:10049000523BC39403EE64809480501390FC9012FE
:1004A00050E312549A1251D070E512529180E0E458
:1004B00090FC86F090FC88F090FC87F090FC89F02E
:1004C00090FC761250E312535A640160030206ADA9
:1004D00090FC791250E312535A60030206AD302F9C
:1004E00002FF2290FC761250E3F990008312177FEE
:1004F000FF54C0440190FC86F06F60031252341226
:100500005540707712536190FC761250E312518976
:10051000400302059B125126FF54E06440704A12CA
:1005200051FC12542712546D90FC7FF090FC81E036
:10053000D3125191506590FC87E0FFC3943C502446
:1005400090FC761250E31254E8EE1252A6FE90FC94
:100550008A1250E3F98F82758300EE1217BE90FC69
:1005600087E004F012542780C390FC761250E31207
:10057000511B12512E12524402050790FC76125064
:10058000E3F990008412177F541F6406600312522F
:100590003412525E1250E3F912AB8212536190FC96
:1005A000761250E31251895052125126FF54E064E2
:1005B0002070361251FC12542712546D90FC7FF0BB
:1005C0001253AFFED39F503390FC88E0C3942D505C
:1005D0001212506A1251E61252C01250E312530620
:1005E0001254A31254F90205C090FC761250E31283
:1005F000511B12512E12524402059E12536190FC5F
:10060000761250E3125189506C125126FF54E06467
:100610008070501251FC90FC7F1251101253461200
:100620005131FF90FC901250E3F9EF1252DB12505F
:10063000E312511BFF04F0E92F125131FF90FC909F
:100640001250E31253A790FC761250E312511BFF95
:1006500004F0E92F125131FF90FC901250E3125434
:100660002E801290FC761250E312511B12512E1262
:1006700052440205FE12527F1250E3F912B121904A
:10068000FC761250E31255321250E3F97E007F805F
:1006900012174090FC761250E31254AB1252349071
:1006A000FE3AE060030211A1D22F0211A190FC7961
:1006B0001250E312535A6401600302115412521192
:1006C00012523BC39480EE64809480501690FC7963
:1006D0001250E3F974801254631251C970E212523D
:1006E0009180DD90FE39E0605390FC761250E32457
:1006F0000012539F54FD1252DB1250E31254AB12FE
:10070000523490FC791250E312524F1250E31216F9
:100710005A1250E3F912B0EC90FC901250E31254CC
:10072000EF1250E31252701250E3F912B12190FE11
:100730003AE060030211A1D22F0211A1302F037FF2
:10074000002290FC761250E312548930E12B1253B0
:100750009D54FD1217AC90FC791250E31254E8C07E
:1007600003C002C00190FC761250E324801252FDB7
:10077000D001D002D00312522D90FC791250E39098
:1007800000831253DA1250E3F990008312177FFEB0
:100790005F54F0444190FC86F06E600312523412B4
:1007A000554060030208A012536190FC761250E39A
:1007B0001251895059125126FF54E06440703D9007
:1007C000FC7FE0FEEF541FFFEE2F90FC818027128C
:1007D00053AFFED39F50D390FC761250E3125127B3
:1007E000FF90FC8A1250E3F990FC87E0F5821253E7
:1007F0003F90FC87E004F012542780D390FC7612DF
:1008000050E312511B12512E1252440207AA1254E5
:100810003690FC791250E31251EEC39F4003020957
:10082000AC12521C6440706C90FC80125204125343
:10083000C212550150DBE412521512516A502412B3
:1008400051AC1250E31251E6547FFF90FC8A1250D3
:10085000E3125181547F6F600A1251D070DC125242
:100860009180D790FC8712538A40231251AC1250CA
:10087000E31251E6FF90FC8A1250E3F990FC87E006
:10088000F58212533F90FC87E004F0125234125567
:100890000D0208311251AC1250E3125199020811A5
:1008A00012536190FC761250E31251894003020901
:1008B000AC12512654E06440600302099A12543687
:1008C00090FC791250E31251EEC39F40030209AC31
:1008D00012521C6440600302098E12532A90FC7667
:1008E0001250E312511B1252A51253B9A3E004F0A7
:1008F00090FC7EE0FFE41254721253AFD39F40038A
:100900000209AC90FE3BA3E090FC7EF090FC80E0FE
:100910001251F5D39F504490FC761250E312511BB4
:100920001252A61253C91250E3125181FE547F6F26
:10093000702390FC87E0C3943C501A90FC761250D0
:10094000E312511B1252A64EFF90FC8A1250E39004
:10095000FC871253381253C202090C90FC87E0FF47
:10096000602390FC761250E312511B1252A6FEEF48
:1009700024FFFDEC34FFFC90FC8A1250E3125181FD
:100980006E600580001252341254270208F9125189
:10099000AC1250E31251990208C090FC761250E359
:1009A00012511B12512E1252440208A390FE3AE03B
:1009B000FF64016008EF64036003020C9612536148
:1009C00090FC761250E31251895042125126FF5486
:1009D000E0642070261251FC1254271253AFFED34C
:1009E0009F50DD12506A1251E61252C01250E312AB
:1009F00053061254A31254F90209DB90FC761250EC
:100A0000E312511B12512E1252440209C0125436E5
:100A100090FC791250E31251EEC39F4003020BD2B7
:100A200012521C64206003020BC612532A1253C2D6
:100A300012550150DBE412521590FC8812516D40A2
:100A400003020B6E1251AC1250E31251E65478FFC0
:100A500090FC8D1250E3125181FE54786F600302B6
:100A60000B6190FC7EE012529B1250E312518154B4
:100A700007FFEE5407FED39F4004AF06800090FCB2
:100A80007EE012529B1250E312518154784FFF9036
:100A9000FC8D1250E3F990FE3BE0FCA3E0FDF582F3
:100AA0008C83EF1217BE90FC7EE024811251B212AB
:100AB00050E31251E6FF90FC8D1250E3F9ED240152
:100AC000FDE43CFC8D82F58312177F4F8D828C8371
:100AD0001217BE12523BF5828E8312177F5478FD97
:100AE000BD013690FC8D1250E3F9EF2402FFE43E85
:100AF000FEE92FF9EA3EFAC003C002C001121766F0
:100B000012545B12529D1250E31251814FD001D00A
:100B100002D0031217AC020B6E90FC7EE090FC79C1
:100B20001250DD1251E6FF90FC8D1250E3F990FE59
:100B30003CE02402FD1253ECFC8D82F58312177FFA
:100B4000FED39F4004AF06800D12545C1251B212C6
:100B500050E31251E6FF90FC8D1250E312530680D1
:100B60000D90FE3CE024031253EBF0020A3990FC96
:100B70008812538A404A1254D390FC791250E312DF
:100B80005181FD90FC8D1250E31254BC1255151288
:100B900050E31251E6FF90FC88E024011252C71284
:100BA00050E312530612545C1251B21250E3125128
:100BB000E61252C01250E31253061254A3125234DA
:100BC00012550D020A301251AC1250E31251990223
:100BD0000A1012536190FC761250E31251894003BF
:100BE000020ED112512654E064806003020C84127C
:100BF000543690FC791250E31251EEC39F40030229
:100C00000ED112521C6480706F12532A90FC76121F
:100C100050E31250EB1253461251311251F504F0C9
:100C20001253CC1250E31251814FFF90FC9012509E
:100C3000E3F9EF1252DB1250E312511B125346122A
:100C400051311251F51252981250E31251814FFF57
:100C500090FC901250E31253A790FC761250E312CE
:100C6000511B1253461251311251F5125298125023
:100C7000E31251814F020EA71251AC1250E31251F0
:100C800099020BF290FC761250E312511B12512E76
:100C9000125244020BD512536190FC761250E312AB
:100CA00051894003020E04125126FF54E064206073
:100CB00003020DF21251FC1254271253AFD39F506E
:100CC000D812543690FC791250E31251EEC39F4073
:100CD00003020DEC12521C64206003020DE012535B
:100CE0002A1253C290FC80E01251F5D39F50D59048
:100CF000FC761250E312511B1252A61253C9125025
:100D0000E3125181547F6F6003020DA990FC88E0CB
:100D1000C3942D4003020DA91254D3125182FD90A9
:100D2000FC8D1250E31254BC90FC7FE02481FDE462
:100D300033FC90FC761250E3125181FD12551512CE
:100D400050E31251E65DFF90FC88E0FE2401125250
:100D5000C71250E31253068E8275830012177F5418
:100D600078640170161250D61251E612545B12527A
:100D70009D1250E31251815FFF80221250D6125112
:100D8000E612545B12529D1250E3125181FEC39F32
:100D90005004AF0680071250D61251E6FF1252C11E
:100DA0001250E31253061254A390FC88E0FF602710
:100DB00090FC761250E312511B1252A6547FFEEFA4
:100DC00024FDFDEC34FFFC90FC8D1250E3125181A8
:100DD000547F6E6005800012523412550D020CE4EF
:100DE0001251AC1250E3125199020CC41254F90280
:100DF0000CBA90FC761250E312511B12512E125273
:100E000044020C9912536190FC761250E3125189FE
:100E10004003020ED112512654E064806003020E9A
:100E2000BF12543690FC791250E31251EEC39F402A
:100E300003020ED112521C6480707812532A90FC67
:100E4000761250E31250EB1253461251311251F503
:100E500004F01253CC1250E31251815FFF90FC90CA
:100E60001250E3F9EF1252DB1250E312511B1253EE
:100E7000461251311251F51252981250E31251811B
:100E80005FFF90FC901250E31253A790FC76125033
:100E9000E312511B1253461251311251F51252985E
:100EA0001250E31251815FFF90FC901250E31254F4
:100EB0002E801E1251AC1250E3125199020E249052
:100EC000FC761250E312511B12512E125244020EA4
:100ED0000712536190FC761250E3125189400302CD
:100EE00011A112512654E0646060030211421254B1
:100EF0003690FC791250E31251EEC39F4003021169
:100F0000A112521C6460600302113612532A90FC35
:100F1000761250E312511B1252A51253B9A3E004EA
:100F2000F01255406003020FF9A3F0A3F0125368CA
:100F300040081253F340030210CC90FC89E0C394A4
:100F40000C4003020FEE12523BC39405EE648094F2
:100F500080402B90FC761250E312511BFD7C00EF79
:100F60002DFFEC3E1252EF90FC7EE02480FDEC124F
:100F700051581250E31251816F60031252341252D1
:100F80003B64064E6018EF64084E6012EF64094E31
:100F9000600CEF640A4E6006EF640B4E703390FCF9
:100FA000761250E312511B1251381250E312518144
:100FB000FEEFD39E400F90FC761250E312511B12AD
:100FC00052E2020FE512540D1250E31251E6FF8077
:100FD0001490FC761250E312511B1251381250E358
:100FE0001251814FFF90FC931250E312533512516E
:100FF000D07003125291020F2DE412521512536851
:1010000040030210CC1253F340030210CC90FC8931
:10101000E0C3940C40030210C112523BC39405EE8E
:1010200064809480402B90FC761250E312511BFD9B
:101030007C00EF2DFFEC3E1252EF90FC7EE024800E
:10104000FDEC1251581250E31251816F600312529D
:101050003412523B64064E6018EF64084E6012EF83
:1010600064094E600CEF640A4E6006EF640B4E702C
:101070003390FC761250E312511B1251381250E398
:10108000125181FEEFC39E500F90FC761250E31276
:10109000511B1252E20210B812540D1250E31251B9
:1010A000E6FF801490FC761250E312511B12513867
:1010B0001250E31251815FFF90FC931250E31253E0
:1010C000351251D07003125291020FFD90FC931211
:1010D00050E3F974031255391250E3F912530FE437
:1010E0001217BE12552050037405F090FC89E0C31E
:1010F0009407402F90FC931250E32405F9E43AFA48
:1011000012176654BF1255391250E3F990000612B7
:10111000177FFFC3942D500280027F2D900006EFB1
:101120001217BE90FC81E00490FC7FF0A3E00490D5
:10113000FC7EF00211A11251AC1250E3125199023F
:101140000EF190FC761250E312511B12512E1252E6
:1011500044020ED490FC761250E3240012539F54A4
:10116000FD1252DB1250E31254AB12523490FC7950
:101170001250E312524F1250E312165A1250E3F972
:1011800012B0EC90FC901250E31254EF1250E312A4
:1011900052701250E3F912B12190FE3AE07002D27F
:1011A0002F90FC961250E3F9121766FF90FC76120E
:1011B00050E3F9900023EF1217BE90FC961250E313
:1011C0001253D71250E3F9900024EF1217BE90FC8F
:1011D000961250E3F99000021253DB1250E3F9909B
:1011E0000025EF1217BE12535B640160030215AFB6
:1011F00090FC87E0C39401500A12525E1250E3F94A
:1012000012AB8290FC88E0C39403501890FDBD742B
:1012100001F0A374FCF0A37488F090FC8D1250E3ED
:10122000F912B0EC125520500A12527F1250E3F915
:1012300012B121E490FC7CF07009D31255214003D7
:101240007405F0E490FC7FF090FC761250E31251AC
:101250001B125346F9EE3AFA74021252DB1250E3B3
:1012600012511BFF04F0E92FF9EE3AFA740312173A
:10127000AC90FC87E0240BFFA3E02FFFA3E02FFF3F
:1012800090FC761250E312511B1251D790FC86E06D
:10129000FF90FC761250E312511BFE04F0EE125147
:1012A000DD90FC87E04440FF90FC761250E3125141
:1012B0001BFE04F0EE1251DDE412521512516A5079
:1012C0002090FC8A1250E3125181FF90FC7612505C
:1012D000E312511B1251D71251D070E0125291807B
:1012E000DB90FC88E04420FF90FC761250E3125122
:1012F0001B1251D7E412521590FC8812516D5020E8
:1013000090FC8D1250E3125181FF90FC761250E355
:1013100012511B1251D71251D070DD12529180D848
:1013200090FC761250E312511B125346F9EE3AFA32
:1013300074831254F21250E3F9121766FF90FC7690
:101340001250E312511B1251D790FC901250E3122D
:1013500053D71250E312511BFE04F0EE1251DD90F0
:10136000FC901250E3F99000021253DB1250E3128A
:10137000511BFE04F0EE1251DD90FC89E04460FF49
:1013800090FC761250E312511BFE04F0EE1251DD78
:10139000E412521590FC8912516D502090FC93126A
:1013A00050E3125181FF90FC761250E312511B1250
:1013B00051D71251D070DD12529180D8E490FC8246
:1013C000F0A304F0A304F0E412521512516A400392
:1013D00002145190FC8A1250E3125181FE547F9006
:1013E000FC85F0EE30E75F1254B4505A90FC85E073
:1013F000FFC3943C505090FC82E004F0E0B4012321
:101400001252B0C003C002C00190FC761250E32417
:10141000361252FDD001D002D00312534E90FC83FD
:10142000F0802390FC85E01252B1C003C002C001DD
:1014300090FC761250E31252FBD001D002D003127E
:10144000534E90FC84F01251D0700312529102134B
:10145000CB90FC82E0C394015030E004F090FC8A11
:101460001250E3F9121766547F1252B1C003C00242
:10147000C00190FC761250E324361252FDD001D008
:1014800002D00312534E90FC83F01254B45060E427
:1014900012521512516A505790FC8A1250E31251A1
:1014A00081547F90FC85F064026005E06403703431
:1014B0001254B4502F90FC85E0FFC3943C5025900B
:1014C000FC82E004F01252B0C003C002C00190FCE4
:1014D000761250E31252FBD001D002D00312534EC9
:1014E00090FC84F01251D0700312529102149312A6
:1014F00054B45019E004F090FC761250E31252FB01
:101500007BFF7A4B794412534E90FC84F0E41252E4
:101510001512516A506C90FC7FE0C3946E5063903A
:10152000FC8A1250E3125181547FFF90FC85F090A9
:10153000FC83E06F6041A3E0FFA3E0FE6F6038EE44
:1015400064016033EEC3943C502DE01252B1C003ED
:10155000C002C00190FC761250E312511B7E00299C
:10156000F9EE1252FFD001D002D0037F12121740C1
:1015700090FC7FE02412F01251D0700312529102BD
:10158000151190FC7FE0FFFDC374809DFDE4940085
:10159000FCC004C00590FC761250E31254E8EF7CC6
:1015A0000029F9EC3AFA7D00D007D00612206090AD
:1015B000FC761250E3F9E41252DB1250E3F974FFA7
:1015C00012552874FF1217BE90000374FF125323A4
:1015D00074FF1217BE90000574FF1217BE9000062C
:1015E00074FF1217BE90000712520C12523B125495
:1015F00052501390FC761250E31251E61251C9700A
:10160000EA12529180E512547A90FC761250E3F976
:1016100090007FEF1217BE12535B6401703690FC8E
:10162000761250E3F99000FE12520C12523B125403
:1016300052501090FC761250E31251BA70ED1252D3
:101640009180E812547A90FC761250E3F99000FFF2
:10165000EF1217BE90FC7DE0FF22F912AB8290FDE5
:10166000BD7401F0A374FCF0A37488F090FC8D228B
:102B570049646C65005472616E736D69745F4D658D
:102B67007373616765005365745F4C6F6769636171
:102B77006C5F4164647265737300436F6E6E656367
:102B87007400446973636F6E6E6563740053746198
:102B97006E646279005374616E6462795F416C6C34
:102BA700005265636F72645F43757272656E74007D
:102BB7005265636F72645F43757272656E745F4FBF
:102BC7006666005365745F54696D65725F50726F16
:102BD7006772616D00436C6561725F54696D657200
:102BE7005F50726F6772616D004765745F4D656E08
:102BF700755F4C616E677561676500416E6E6F75D5
:102C07006E63655F4D656E755F4C616E6775616775
:102C17006500436F6E74726F6C5F4465636B00533E
:102C2700656C6563745F54756E65725F5365727624
:102C370069636500436F6E74726F6C5F54756E6580
:102C4700720053656E645F56656E646F725F436FA3
:102C57006D6D616E640042726F6164636173745F6E
:102C670056656E646F725F436F6D6D616E6400567B
:102C7700656E646F725F52656D6F74655F427574E0
:102C8700746F6E5F507265737365640056656E642A
:102C97006F725F52656D6F74655F427574746F6EA6
:102CA7005F52656C65617365640052657175657324
:102CB700745F4D656E7500557365725F436F6E7413
:102CC700726F6C5F507265737365640055736572DC
:102CD7005F436F6E74726F6C5F52656C656173658D
:102CE7006400526571756573745F53797374656DAC
:102CF7005F417564696F5F4D6F646500557064610E
:102D070074655F4465766963655F496E666F0052F7
:102D17006571756573745F496D6167655F56696550
:102D2700775F4F6E00526571756573745F54657890
:102D3700745F566965775F4F6E00416E6E6F756E93
:102D470063655F4163746976655F536F7572636529
:102D5700005365745F496E6163746976655F536F8D
:102D67007572636500526571756573745F44697345
:102D7700706C61795F4F53445F537472696E67007B
:102D8700496E666F726D5F4D656E755F53746174E2
:102D97007573005365745F53797374656D5F41751F
:102DA70064696F5F4D6F6465005265706F72745F21
:102DB7005265636F72645F53746174757300526513
:102DC700706F72745F54696D65725F537461747567
:102DD70073005265706F72745F54696D65725F43FB
:102DE7006C65617265645F53746174757300556EC9
:102DF700737570706F727465645F4D657373616727
:102E07006500496D6167655F566965775F4F6E005D
:102E1700546578745F566965775F4F6E00416374D8
:102E27006976655F536F7572636500496E61637498
:102E37006976655F536F7572636500526571756575
:102E4700737465645F666F725F5374616E646279F1
:102E570000496E666F726D65645F4D656E755F4C98
:102E6700616E67756167650052656365697665645C
:102E77005F56656E646F725F436F6D6D616E640060
:102E870052656365697665645F56656E646F725FE8
:102E970052656D6F74655F427574746F6E5F5072C3
:102EA70065737365640052656365697665645F562B
:102EB700656E646F725F52656D6F74655F4275749E
:102EC700746F6E5F52656C65617365640044697306
:102ED700706C61795F4F53445F537472696E67001A
:102EE700496E666F726D65645F4D656E755F53748D
:102EF700617475730052656365697665645F5573C0
:102F070065725F436F6E74726F6C5F507265737337
:102F170065640052656365697665645F55736572BC
:102F27005F436F6E74726F6C5F52656C656173653A
:102F3700640053797374656D5F417564696F5F4DA4
:102F47006F64655F536574004465766963655F49BF
:102F57006E666F5F4368616E676564005365745F93
:102F670053747265616D5F50617468005265717565
:102F770065737465645F5265636F72645F437572EE
:102F870072656E74005265717565737465645F521E
:102F970065636F72645F43757272656E745F4F66C7
:102FA70066005265717565737465645F5365745F18
:102FB70054696D65725F50726F6772616D0052651B
:102FC700717565737465645F5365745F54696D6586
:102FD700725F50726F6772616D5F5469746C6500E0
:102FE7005265717565737465645F436C6561725F83
:102FF70054696D65725F50726F6772616D005265DB
:10300700717565737465645F666F725F4D656E7524
:10301700005265717565737465645F436F6E747292
:103027006F6C5F4465636B0053656C6563746564BF
:103037005F54756E65725F5365727669636500529A
:1030470065717565737465645F436F6E74726F6CD9
:103057005F54756E6572005265717565737465644A
:103067005F666F725F53797374656D5F41756469ED
:103077006F5F4D6F646500526F7574696E675F4F60
:10308700666600443D307825302E32582044656509
:103097007020436F6C6F7220446574656374656458
:1030A7000D0A00443D307825302E32582034204F09
:1030B700757470757420537570706F72740D0A0093
:1030C700443D307825302E325820547820545245CC
:1030D70047203D20307825302E32580D0A004552C2
:1030E700524F523A204E3D307825302E32582041EB
:1030F7004B535620524459202D204D4355204949C2
:10310700432025640D0A004552524F523A204E3D46
:10311700307825302E325820414B53562072656146
:1031270064202D204D4355204949432025640D0A2D
:10313700004552524F523A204E3D307825302E32BC
:103147005820414B53562072656164202D204B65F2
:10315700792057726F6E670D0A004552524F523AE7
:10316700204E3D307825302E325820547820526931
:103177002072656164202D204D4355204949432025
:1031870025640D0A004552524F523A204E3D307881
:1031970025302E325820424B5356207265616420E9
:1031A7002D20444E204444432025640D0A004552F7
:1031B700524F523A204E3D307825302E3258204219
:1031C7004B53562072656164202D204B657920573B
:1031D700726F6E670D0A004552524F523A204E3DAC
:1031E700307825302E325820527820526920726567
:1031F7006164202D20444E204444432025640D0A59
:10320700004552524F523A204E3D307825302E32EB
:1032170058204B5356204649464F2072656164201B
:103227002D20444E204444432025640D0A00455276
:10323700524F523A204E3D307825302E3258204B8F
:103247005356204649464F2072656164202D204B16
:1032570065792057726F6E670D0A004552524F52BB
:103267003A204E3D307825302E3258204544494487
:103277002062302072656164202D20444E20444432
:10328700432025640D0A004552524F523A204E3DC5
:10329700307825302E32582045444944204368650C
:1032A700636B206661696C65642C207045444944F2
:1032B7005B3132365D3D307825302E3258203E2046
:1032C700380D0A004552524F523A204E3D3078256C
:1032D700302E325820454449442062692072656186
:1032E70064202D20444E204444432025640D0A00C9
:1032F7004552524F523A204E3D307825302E3258A3
:10330700204544494420636865636B73756D206588
:1033170072726F720D0A005741524E494E473A205A
:10332700443D307825302E3258204E6F204550438B
:10333700432064657465637465640A0D00443D3019
:103347007825302E325820455043432064657465F4
:1033570063746564205665723D25642E25640A0DE5
:10336700005741524E494E473A204E6F20446576EA
:1033770069636520666F756E640D0A005741524E8A
:10338700494E473A204E6F20417564696F20537943
:103397007374656D20666F756E640D0A0057415230
:1033A7004E494E473A20443D307825302E3258203A
:1033B70045504343204576656E74204D69737369A4
:1033C7006E670D0A004552524F523A20443D3078FD
:1033D70025302E3258204550434320436F6D6D6191
:1033E7006E642054696D652D6F75740D0A00455222
:1033F700524F523A20494943206661696C656420FF
:1034070025642C20494943416464723D3078253056
:103417002E32582C20526567416464723D307825FE
:10342700302E32580D0A00FF2B57FF2B5CFF2B6DF8
:10343700FF2B81FF2B89FF2B94FF2B9CFF2BA8FFD2
:103447002BB7FF2BCAFF2BDCFF2BF0FF2C02FF2C27
:1034570019FF2C26FF2C3BFF2C49FF2C5DFF2C76F8
:10346700FF2C93FF2CB1FF2CBEFF2CD3FF2CE9FFC1
:103477002D03FF2D16FF2D2CFF2D41FF2D58FF2D5E
:103487006CFF2D87FF2D9AFF2DB0FF2DC5FF2DD97E
:10349700FF2DF5FF2E09FF2E17FF2E24FF2E32FFDB
:1034A7002E42FF2E58FF2E6FFF2E87FF2EADFF2EC9
:1034B700D4FF2EE7FF2EFCFF2F1AFF2F39FF2F4FC8
:1034C700FF2F63FF2F73FF2F8CFF2FA9FF2FC5FF40
:1034D7002FE7FF3005FF3018FF302FFF3046FF3052
:0434E7005EFF307ED6
:0C87EE0001680042FCE000000264000092
:106CA50090FD1DE0FBA3E0FAA3E0F9121766FF9043
:106CB500FD20E0FBA3E0FAA3E022F090FCE6E475FA
:106CC500F001121893FE748025F0F58274FF3EF5ED
:106CD500837469F090FCE6E475F001121893FE7474
:106CE5008025F0F58274FF3EF58322F912176604BC
:106CF500FF90FD977B00E47A007922F0A304F0224F
:106D0500F0A3EDF0A3EBF0A3EAF0A3E9F02212174C
:106D15006604FF90FD4E7B00E47A007922F0A32201
:106D2500F9121766FF90FBCAE4F0A3EFF02290FF7B
:106D350080F090FCF2E47B017AFF7980F0A322F9E0
:106D450090000102177F2407F9E43AFA90FD4EE41A
:106D5500F0A322F9121766FF90FE23E4F0A30422A4
:106D6500F9121766FFE490FE23F0A3227B007A0058
:106D7500792290FCF2E4F0A32290FCE2E090FBCCB7
:106D8500FFE4F0A3EFF022F990FCE6E0FEA3E0F5C6
:106D9500828E8302177FF990000212177FFF900001
:106DA5000312177FFD22F9121766FF7B017AFF791F
:106DB50080227967E7C4F8540FC868FF19E7C454FF
:106DC500F048FEE42FFDEE22F9A3E0FFA3E090FCDE
:106DD500F2CFF0A3EFF0222FF9EA3EFA9000041269
:106DE500177FFF90000512177FFD2290FCE2EFF060
:106DF500E0FE2204F0A3F07D74FF22F990FD97E4F4
:106E0500F0A3222401F9E43AFA021766E490FCE6BD
:106E1500F0A3F0227405F0E4A3F07D757F0122F95B
:106E250012176604FF2290FD38E0FD90FBCAE4F0DE
:106E3500A3EDF0A32290FCE6E0FDA3E090FD4ECD8E
:106E4500F0A3EDF022A3E4F0A3E522F07BFF7A3076
:106E550079C72290FCE6E4F0740AA3F0E4A3F0A35A
:106E6500F02290FCE7E004F02290FCE6E004F0223A
:106E750090FDE3E014FF90FDE2E022D390FCE7E013
:106E8500940090FCE6E064802290FCE9E004F022A6
:106E950090FCE8E004F022C390FCE9E0940390FC48
:106EA500E8E064809480227480F0E4A3F07DA17F03
:106EB500012290FCE2E0FF90FBCC22E025E0FF9070
:106EC500FCE6E033FE90FCEA22C390FE60E094E825
:106ED50090FE5FE0940322A3E024FDF090FCE6E041
:106EE50034FFF02204F0A3F07DA0FF2290FE22E003
:106EF500FF7401A807082290FCE6E0FEA3E0FFC3AB
:106F050022E52225E0F52222F0A37402F07D747FAC
:026F1500012257
:10862A0090FCE3126D0A90FDC9E0F9A3E0FAA3E019
:10863A0090FCEAC9126D0B90FCEA126CB7126D9BA2
:10864A0012781590FCEA126CB7126D9B7B021267C6
:10865A001090FCEA126CB7F9121766FF126D45FD0D
:10866A0012797C90FCEA126CB7F9121766FF126D48
:10867A0045FD7B0112671012ABAF7D087F061278A9
:10868A00157B017D087F06126710126E11126EFCAF
:10869A009407EE64809480501FEF25E0FFEE33FECE
:1086AA0090FCEA126CB7126DDC7B01126710126E35
:1086BA00677003126E6E80D5E4FB7D01FF12AA1764
:1086CA007B02E4FD7F0112AA177BFF7AA0791FE4DF
:1086DA00FF12B2A490FE6474FEF07BA0E4FD12A81F
:1086EA00877BFF7A00794EE4FF12B2937D0102A7DD
:0186FA0091EE
:10ABAF0090FCEA126CB7F9121766FF126D45FD1291
:10ABBF00797C12951290FCEA126CB7F9121766FFA6
:0CABCF00126D45FD1278157F0402B325BD
:10B25A0090FCEA126CB7126D9B1278157D02E4FF1E
:03B26A0002AEE948
:1001EE00E4FDFF12AEE990FCEA126CB7126D9B02B1
:0201FE00797C0A
:1092A00090FE7A126D0A90FE7A126CB7F9ED1217E1
:1092B000AC90FE7A126CB7F9900001E41217BE125E
:1092C0006CF17D0512896690FCE2E07024E5226075
:1092D0002090FE7A126CB7126D257BFF7A30798A66
:1092E00012A49390FE7A126CB7126E0844401217C3
:1092F000AC75220890FE7A126CB7F9121766126CE0
:10930000F57D0712896690FE7A126CB7126CF07DBB
:109310000712896690FCE2E0702330132090FE7AF9
:10932000126CB7126D257BFF7A3079AA12A4939044
:0E933000FE7A126CB7126E0844801217AC223F
:0DB2FF00126D4530E6047F0180027F0022C1
:108E050090FE7D126D0A90FE7D126CB7126D443096
:108E1500E53230E61B30E70D126D66F07B037D060B
:108E250012A608800090FE7D126CB7126D5880392D
:108E350090FE7D126CB7126D58128EAC126CB71283
:108E45006D58803E90FE7D126CB7126D4430E62061
:108E550030E70D126D66F07B037D0612A6088000D3
:108E650090FE7D126CB7126D65F07B067D0680174E
:108E750090FE7D126CB7126D65128EAC126CB71236
:108E85006D65F07B047D0A12A60890FE7D126CB715
:108E9500126CF07D0612896690FE7D126CB7126D1C
:108EA50025126E4A02A493F07B057D0A12A608904E
:038EB500FE7D221D
:10AC5F0090FE80126D0AED90FE80600A126CB712A2
:10AC6F006E0844208008126CB7126E0854DF12175A
:0BAC7F00AC90FE80126CB7F9028E054D
:10A3F80090FE83126D0A90FE83126CB7126D443082
:10A40800E40830E61C126D66800F90FE83126CB76C
:10A41800126D4430E60B126D59F07B077D0612A6CB
:10A428000890FE83126CB7126CF07D061289669054
:0EA43800FE83126CB7126D25126E4A02A493B9
:10AC8A0090FE86126D0AED90FE86600A126CB7126B
:10AC9A006E0844108008126CB7126E0854EF12172F
:0BACAA00AC90FE86126CB7F902A3F814
:10A8FF0090FE89126D0A90FE89126CB7126D44306A
:10A90F00E60B126D59F07B057D0612A60890FE89A5
:10A91F00126CB7126CF07D0612896690FE89126C6C
:0AA92F00B7126D25126E4A02A493C0
:10ABDB0090FE8C126D0A90FE8C126CB7126D443085
:10ABEB00E708126D66F07B03800C90FE8C126CB73D
:0CABFB00126D65F07B017D0712A6082298
:109B9D0090FE8F126D0A90FE8F126CB7126D4430CD
:109BAD00E634752208121766126CF57D051289666A
:109BBD0090FE8F126CB7126D4430E70575228280CE
:109BCD000A75229690FE8F126CB7F9121766126CF9
:109BDD00F57D0612896690FE8F126CB7F9128E050F
:109BED0090FE8F126CB7F912A3F890FE8F126CB71E
:109BFD00126D4430E708126D59F07B03800B90FE17
:0F9C0D008F126CB7126D58F0FB7D0712A608225C
:10AB1F0090FE92126D0A90FE92126CB7126CF07D3D
:10AB2F000712896690FE92126CB7126D4430E708D7
:10AB3F00A216821782138006A21682178211E4339F
:02AB4F00FF22E3
:0EB2D500126CF17D07128966A215E433FF2288
:10B19900126CF17D0712896690FCE2E060037F0181
:07B1A90022A214E433FF228F
:0EB2E300126CF17D08128966A216E433FF2278
:0EB2F100126CF17D40128966A210E433FF2238
:10000E00121766FF90FDCF126CB7126E007403F0DC
:05001E007D500289661F
:10B13900121766FF90FD6B126CB7F9A3E0FD126E52
:08B1490001EDF07D8002896632
:10B1DE0012176604FF90FDD5126CB7126E0074083C
:06B1EE00F07D41028966BC
:10005600121766FF90FDDB126CB7126E007414F077
:050066007D60028966C7
:10B0170090FE95126D0A90FE95126CB7F912A691E3
:10B0270090FE95126CB7126D65F0FB7D0802A608BD
:10AF300090FE98126D0A90FE98126CB7F912A691C5
:10AF400090FE98126CB7126D58F0E4FB7D0802A6D3
:01AF500008F8
:10AF510090FE9B126D0A90FE9B126CB7F912A6919E
:10AF610090FE9B126CB7126D58F07B077D0802A60C
:01AF710008D7
:10AF720090FE9E126D0A90FE9E126CB7F912A69177
:10AF820090FE9E126CB7126D65F07B077D0802A6DB
:01AF920008B6
:10AF930090FEA1126D0A90FEA1126CB7F912A69150
:10AFA30090FEA1126CB7126D58F0E4FB7D0F02A660
:01AFB3000895
:10B0370090FEA4126D0A90FEA4126CB7F912A691A5
:10B0470090FEA4126CB7126D65F0FB7D0F02A60887
:109E7E0090FE3D126D0AA3EDF012A69190FE3D12DA
:109E8E006CB7126CF07D091289663011037F0122C6
:109E9E0090FE40E0FF12A1ACE4F522FB90FCF21222
:109EAE006CFCA3F07D60FF1274FFE4F522FB90FCC6
:109EBE00F2126D1E126EE91274FF126DF0C0069052
:109ECE00FCF2126CF9126EAF1274FFD0E04F90FCE0
:0A9EDE00E2F070037F02227F0022F1
:1000260090FEA7126D0A90FEA7126CB7F912A69160
:1000360090FEA7126CB7126CF07D09128966A212A7
:04004600E433FF227E
:10AFB40090FEAA126D0A90FEAA126CB7F912A6911D
:10AFC40090FEAA126CB7126D58F0E4FB7D0E02A637
:01AFD4000874
:10B0570090FEAD126D0A90FEAD126CB7F912A69173
:10B0670090FEAD126CB7126D65F0FB7D0E02A6085F
:10AFD50090FEB0126D0A90FEB0126CB7F912A691F0
:10AFE50090FEB0126CB7126D58F07B047D0F02A66F
:01AFF5000853
:10AFF60090FEB3126D0A90FEB3126CB7F912A691C9
:10B0060090FEB3126CB7126D65F07B047D0F02A63D
:01B016000831
:10AC070090FD6F126D0A90FD6F126CB7F912A69145
:10AC170090FD6F126CB7F9121766FF90FD73126CF7
:0CAC2700B7126E007408F07D15028966FB
:10A80D0090FE41126D0AA3EDF012A69190FE411239
:10A81D006CB7126CF07D0F12896690FCE2EFF06060
:10A82D00167BFF7A3079E590FE44E0126D29126DAA
:0DA83D007E12A4937F0022A217E433FF22B5
:1090BA0090FD76126D0AA3EDF012A69190FD76123C
:1090CA006CB7126E2490FD7A126CB7126E00740798
:1090DA00F07D1D12896690FCE2EFF060127BFF7A48
:1090EA0031790E90FD79E0126D29126EB78058120F
:1090FA006E11A3F0A3F0F522752201E522601A9001
:10910A00FD7A126CB7126D8C55226008126E8E7041
:10911A0003126E95126F0680E2126E677003126E6A
:10912A006E90FCE6E07004A3E0640570CB90FCE866
:10913A00E07004A3E0641460197BFF7A31793890F7
:10914A00FD79E0FF90FBCAE4F0A3EFF012A4937F4D
:05915A0000227F01224C
:10AC330090FD7D126D0A90FD7D126CB7F912A691FD
:10AC430090FD7D126CB7F9121766FF90FD81126CAF
:0CAC5300B7126E007405F07D10028966D7
:10ACE00090FEB6126D0A90FEB6126CB7F912A691DC
:10ACF00090FEB6126CB7126CF07D0F128966E522D9
:0AAD000030E1047F0180027F002291
:10A5C20090FD84126D0AA3EDF012A69190FD841203
:10A5D2006CB7126E2490FD88126CB7126E00740272
:10A5E200F07D2212896690FCE2EFF060167BFF7A22
:10A5F20031796190FD87E0126D29126D7E12A4936C
:06A602007F00227F01220F
:10AD0A0090FD8B126D0A90FD8B126CB7F912A69109
:10AD1A0090FD8B126CB7126E2490FD8F126CB712D5
:0AAD2A006E007408F07D25028966B2
:108D480090FE46126D0A90FE45EFF012A1AC90FE1F
:108D580046126CB7F9E41217AC90FE46126CB7F9DC
:108D6800126D77126DF81274FF126DF0C00690FE46
:108D780046126CB7F9126D77126E191274FFD0E0B3
:108D88004F90FCE2F060127BFF7A31798C90FE45BF
:108D9800E0126D29126EB78056126E11A3F0A3F07F
:108DA800752201E522601A90FE46126CB7126D8C8E
:108DB80055226008126E8E7003126E95126F06802F
:108DC800E2126E677003126E6E90FCE6E07004A308
:108DD800E0640570CB90FCE8E07004A3E0641460E4
:108DE800197BFF7A3179B590FE45E0FF90FBCAE424
:0D8DF800F0A3EFF012A4937F00227F012270
:10B0770012A1AC75224090FCF2126D1B126DF812F2
:0FB0870074FF126D7104126E1B1274FFAF222240
:10AD880090FEF4EDF012A1AC752215126D71126DE2
:10AD9800F81274FF7B017AFE79F4126D7704F0A340
:09ADA80004F07D747F010274FFC8
:10ADDA0090FEB9126D0A12A1AC752218126D711289
:10ADEA006DF81274FF90FEB9126CB7F9126D777490
:07ADFA0008126F0D0274FF47
:10AE010090FEBC126D0A12A1AC752210126D711266
:10AE11006DF81274FF90FEBC126CB7F9126D777465
:07AE210005126F0D0274FF22
:10A0850090FE4A126D0A90FE49EFF012A1AC90FEC7
:10A095004A126CB7F974081217AC90FE4A126CB7E5
:10A0A500F9126D77126DF81274FF126DF0C00690FB
:10A0B500FE4A126CB7F9126D777402126E1B127498
:10A0C500FFD0E04F90FCE2F060167BFF7A3179DE3D
:10A0D50090FE49E0126D29126D7E12A4937F002235
:03A0E5007F0122D6
:10A9730090FEBF126D0A12A1AC90FEBF126CB7F924
:10A9830074411217AC90FEBF126CB7F9126D7712B7
:10A993006DF81274FF90FEBF126CB7F9126D7774E5
:07A9A30002126E1B0274FF9B
:10A9AA0090FEC2126D0A12A1AC90FEC2126CB7F9E7
:10A9BA0074201217AC90FEC2126CB7F9126D77129E
:10A9CA006DF81274FF90FEC2126CB7F9126D7774AB
:07A9DA0014126E1B0274FF52
:107EDA0090FDDF126D0A90FDDEEFF012A1AC90FD6D
:107EEA00E2E0703B752243FB7A00792290FCF2F0C3
:107EFA00A3126DF81274FF126E7590FDDFB5070CB0
:107F0A00126CB7F9126D77126E19803D126CB7F9BF
:107F1A00126D777405F0A37401F07D75FF802A1243
:107F2A006E7590FDDFB5070F126CB7F9126D777495
:107F3A0005F0A37402800D126CB7F9126D777405FF
:107F4A00F0A37403F07D757F011274FF90FCE2EFD9
:107F5A00F090FCE2E0FF60177BFF7A32790890FD2F
:107F6A00DE126E2EE4F0A3EFF012A4937F00221229
:107F7A006E11A3F0A3F0752201E522601A90FDDFCD
:107F8A00126CB7126D8C55226008126E8E70031235
:107F9A006E95126F0680E2126E677003126E6E9013
:107FAA00FCE6E07004A3E0640570CB90FCE8E070A6
:107FBA0004A3E0641460327BFF7A32793590FDDEE7
:107FCA00E0126D2912A493126E756F601990FDDF8D
:107FDA00126CB7F9E490FCF2F0A3F0A37402F07DFE
:0C7FEA00757F011274FF7F00227F0122CE
:1071430090FD39126D0A90FD38EFF012A1ACE49076
:10715300FF80F090FCF2126D3B127337E490FF80D6
:10716300F0126DB090FCF2F0A3126EE91274FF12EC
:107173006DF0C00690FD39126CB7F9126D77126E7F
:10718300AC1274FFD0E04F90FCE2F060137BFF7A07
:1071930032796290FD38E0126D29126EB70272796E
:1071A30090FD39126CB7F990007E12177FFFD394CC
:1071B300084014126E2BE4F0A3EFF07BFF7A3279D0
:1071C3008E12A4937F052290FD39126CB7F99000BB
:1071D3007E12177F90FD3DF090007EE41217BEE40F
:1071E30090FD3EF090FD3C04F090FD3DE0FF90FDEE
:1071F3003CE0FED39F4003027290EEC313126D3343
:1072030012733790FD3CE05401C43333335480127E
:107213006D33126EE91274FF126DF0C006126D37F2
:10722300126EAC1274FFD0E04F90FCE2F090FF803E
:10723300E06402703190FD3EE0702B04F090FD3964
:10724300126CB72480F9E43AA801FCAD03126DB0C7
:107253007E007F8012174090FD39126CB7F99000C1
:107263007E74011217BE90FCE2E0FF60177BFF7A89
:107273003279CB126E2BE4F0A3EFF012A49390FCBF
:10728300E2E0FF2290FD3CE004F00271EC90FD3956
:10729300126CB7F9E41217AC90FD39126CB7F99080
:1072A300000174FF1217BE90000274FF1217BE9004
:1072B300000374FF1217BE90000474FF1217BE90F0
:1072C300000574FF1217BE90000674FF1217BE90DC
:1072D3000007E41217BEE490FD3FF0126E1290FD1A
:1072E3003EE060067E017F0080047E007F80C390C5
:1072F300FCE7E09FEE6480F8126E8798501A90FDC9
:1073030039126CB7126D8CFF90FD3FE02FF0126EB7
:107313006770CB126E6E80C690FD3FE060137BFFFB
:107323007A3279F790FD38E0126D2912A4937F0623
:0F733300227F002204F0A3F07D60FF1274FF227E
:109D8F0090FEC5126D0AED1217AC90FEC5126CB79E
:109D9F00126E2490FD4E126D3A7402F07D007C0419
:109DAF001286FB90FCE2EFF090FEC5601C126CB7C0
:109DBF00126D257BFF7A33791E12A49390FEC51284
:109DCF006CB7F9900001E4802B126CB7126D2590DF
:109DDF00FF80126D8190FF81E090FBCE126D857B2D
:109DEF00FF7A33794412A49390FEC5126CB7F990A1
:089DFF00000174011217BE22DD
:1081DD0090FE4D126D0AA3EDF090FE4D126CB74A54
:1081ED004B70030282C490FE4D126CB7126D442089
:1081FD00E0030282C4126E1190FCE6126CDD741263
:10820D00126CD874DE126CD8740FF0126DAC126E45
:10821D003A7D027C011286FB126E1190FE50E0FF3A
:10822D0090FCE6E475F001121893FC748025F0F5CE
:10823D008274FF3CF583EF126CD874FF126CD8E496
:10824D00F090FCE6126CDD7463126CD87468126CDD
:10825D00BF7445126CD87458126CD87450126CD807
:10826D007445126CD87450126CD8742D126CD8746D
:10827D0053126CD87470126CD8746C126CBF747409
:10828D00126CD87474126CD87465126CD874721226
:10829D006CD8E4F090FCE6126CDDE4F090FCE61294
:1082AD006CDDE4F090FE4D126CB7126DAB126E3AB0
:0882BD007D097C011286FB2201
:10A25D0090FE51126D0AA3EDF090FE51126CB74AAB
:10A26D004B604190FE51126CB7126D4430E03512C7
:10A27D001766FF7D0412A14A90FE54E0F52290FE70
:10A28D0051126CB7F9121766126D1704F07D007C30
:10A29D00051286FB90FE51126CB7F9121766FF7D01
:05A2AD000312A14A228A
:10AA4D0090FDE4126D0A90FDE4126CB74A4B602440
:10AA5D0090FDE4126CB7126D4430E018121766FFCA
:10AA6D0090FDE7126CB7F9126D517402F07D077C01
:05AA7D00011286FB221E
:107DA10090FD1D126D0A90FD1D126CB74A4B7003B8
:107DB100027EC390FD1D126CB7126D4420E00302D8
:107DC1007EC3126CB4F912176624FE6074146071DC
:107DD10014600D147003027EA424046003027EC3A8
:107DE10090FD23126CB7F9121766601DEA494B60CA
:107DF1001890FD1D126CB7F9121766FF90FD231242
:107E01006CB7F9126D51127EC4126CA5F9126D5145
:107E110004F07D09FC1286FB126CA52403126D4D42
:107E2100127ECF126CA52406126D4D04F07D0BFC61
:107E31001286FB126CA5126D4B04F07D28FC027EAC
:107E4100C090FD23126CB7F9121766601DEA494B09
:107E5100601890FD1D126CB7F9121766FF90FD2393
:107E6100126CB7F9126D51127EC4126CA5F9126D24
:107E71005104F07D09FC1286FB126CA52403126DDE
:107E81004D127ECF126CA52406126D4D04F07D0BB0
:107E9100FC1286FB126CA5126D4B7408F07D297CD7
:107EA10001801C126CA5F9126D5104F07D0AFC12BF
:107EB10086FB126CA5126D4B7402F07D317C0112B0
:107EC10086FB22740EF07D127C011286FB22740364
:097ED100F07D0F7C011286FB22FA
:10AA820090FDEA126D0A90FDEA126CB74A4B6024FF
:10AA920090FDEA126CB7126D4430E018121766FF8F
:10AAA20090FDED126CB7F9126D517403F07D0C7CC0
:05AAB200011286FB22E9
:10A7520090FD40126D0A90FD40126CB74A4B700397
:10A762007F012290FD40126CB7126D4420E0037FFE
:10A77200012212176604FF90FD43126CB7F9A3126F
:0FA782006E3D7D007C071286FB90FCE2EFF0221B
:108A300090FD26126D0A90FD26126CB74A4B70020B
:108A4000FF2290FD26126CB7126D4420E0037F00D8
:108A500022786676000876017866E6FE08E6FFC3AF
:108A6000940FEE94004003028AEDEF64054E606FB0
:108A700090FD26126CB7126E24C007126DB7340237
:108A8000FC126D1804F0D0071286FBE522F4604F4B
:108A9000E522604B90FD26126CB7126E24C00712BF
:108AA0006DB73402FC90FD29126CB7F9126D517448
:108AB0000FF0D0071286FB90FD26126CB7126E24C1
:108AC000C007126DB73403FC90FD2C126CB7F9127D
:108AD0006D51740EF0D0071286FB7867E6FF22789E
:108AE0006706E6186003028A5806028A587BFF7AF6
:098AF00033796812A4937F00227F
:10A0E80090FDF0126D0A90FDF0126CB74A4B7002A9
:10A0F800FF2290FDF0126CB7126D4420E0037F0040
:10A1080022126D1304F07D507C021286FBE522F4C6
:10A118006024E522602090FDF0126CB7126E249046
:10A12800FDF3126CB7F9126D517409F07D507C0281
:10A138001286FB7F05227BFF7A33798312A4937FF3
:02A148000022F3
:10A9E10090FDF6126D0A90FDF6126CB74A4B602588
:10A9F10090FDF6126CB7126D4430E019121766041F
:10AA0100FF90FDF9126CB7F9126D51740FF07D00D2
:06AA11007C021286FB220C
:109D160090FE55126D0AA3EDF090FE55126CB74AEF
:109D26004B605A90FE55126CB7126D4430E04EE40B
:109D360090FF80F0126DAC126D5104F0FDFC12869E
:109D4600FB90FF8074FF126E6090FE55126CB71286
:109D56006DAB126D51129D847F0112B33190FF805D
:109D66007405F090FE58E090FF81F0E4A3F090FEB9
:109D760055126CB7126DAB126D51129D842274038D
:099D8600F07D207C011286FB2215
:10AAB70090FDFC126D0A90FDFC126CB74A4B6024A6
:10AAC70090FDFC126CB7126D4430E018121766FF48
:10AAD70090FDFF126CB7F9126D517408F07D207C60
:05AAE700011286FB22B4
:109EE80090FD2F126D0AA3EDF090FD2F126CB74A6A
:109EF8004B605690FD2F126CB7126D4430E04A1239
:109F08001766FF7B017AFD7932126D5104F0FDFC72
:109F18001286FB90FD2F126CB7F9121766FF90FDA1
:109F280035126CB7F990FD34E0FD126D51EDF07DFE
:109F3800007C051286FB90FD2F126CB7F91217668C
:0A9F4800FF90FD33E0FD12A14A2254
:109A920090FEC8126D0A90FEC8126CB74A4B700253
:109AA200C32290FEC8126CB7126D4420E002C3229A
:109AB200D390FCE1E0942090FCE0E064809480404C
:109AC2001C90FEC8126CB7126D257BFF7A3379A405
:109AD20012A493E490FCE0F0A3F07868F67868E6CC
:109AE200603290FEC8126CB7F9126D1304F07D0556
:109AF200FC1286FB30110F7868E6600116E490FCD8
:109B0200E0F0A3F0D32290FCE1E004F0700690FCB8
:069B1200E0E004F0C322B4
:10A1AC0090FEF5EFF0126E11126EFC9406EE6480C8
:10A1BC009480504274047E00A807088005C333CEF7
:10A1CC0033CED8F9FF90FEF5E0FDEF5D90FCE76033
:10A1DC000E126EC0126CB7126DDC127815800C1258
:10A1EC006EC0126CB7126DDC12797C126E67700344
:0BA1FC00126E6E02A1B47F0102B319C5
:10A6910090FE5CEDF090FE59126D0A126CF17D078F
:10A6A10012896690FE59126CB7126D4490FE5C30AF
:10A6B100E70AE05403FFE52254FC8008E05401FF5F
:10A6C100E52254FE4FF522121766126CF57D070242
:02A6D100896698
:10A6080090FE22EBF090FE20EFF0A3EDF0EF126C3D
:10A61800F412896690FE23E07002A3E0600D126ECA
:10A62800F18002C333D8FC4222800C126EF1800202
:10A63800C333D8FCF4522290FE20E0FFA3E0FD12C1
:05A648006CF6028966BA
:10A14A0090FE5DEFF0ED126E5F90FE5DE0126D160F
:10A15A0004F07D06FC1286FBEF7004E52260187F8E
:10A16A000112B33190FE60E004F0700690FE5FE0E9
:10A17A0004F0126ECE40D2126ECE40107BFF7A33BC
:10A18A0079CC90FE5DE0126D2912A49390FE5DE0F9
:10A19A00FF7B017AFE795E126D5104F07D06FC02A6
:02A1AA0086FB32
:1089660090FD92EF126D05126E5890FD92E030E088
:108976002614FD7B017AFD7993126D77128A2612F1
:108986006DF0C00690FD92E0FD90FD94126CB7125A
:108996006DCDE4A3F0802990FD92E0FD7B017AFD88
:1089A6007993126D77128A26126DF0C00690FD92A9
:1089B600E0FD90FD94126CB7126DCDA37402F0E445
:1089C600FF1274FFD0E04F90FCE2F090FCE2E06012
:1089D6002390FCE6A3E0FF12B325126E809480403C
:1089E60003126EDC126E8E7003126E95126E9C5020
:1089F6000302897090FCE2E0FF601F7BFF7A337907
:108A0600F5126D2A90FD92126D8190FD93E0FF9014
:108A1600FBCEE4F0A3EFF012A49390FCE2E0FF2279
:0A8A260004F0A3F0E4FF1274FF2235
:1086FB0090FD48EFF0A3EC126D05126E5890FD48FB
:10870B00E030E02614FD7B017AFD7949126D77127A
:10871B0087C0126DF0C00690FD48E0FD90FD4B1236
:10872B006CB7126DCDE4A3F0802990FD48E0FD7B82
:10873B00017AFD7949126D771287C0126DF0C00670
:10874B0090FD48E0FD90FD4B126CB7126DCDA374FC
:10875B0002F0E4FF1274FFD0E04F90FCE2F090FCCB
:10876B00E2E0602390FCE6A3E0FF12B325126E80DB
:10877B0094804003126EDC126E8E7003126E951293
:10878B006E9C500302870890FCE2E0FF60217BFFA8
:10879B007A3379F5126D2A90FD48126D8190FD495F
:1087AB00E0FFA3E090FBCECFF0A3EFF012A49390E9
:1087BB00FCE2E0FF227402F0A314F0E4FF1274FF5A
:0187CB00228B
:10A01F0090FEE6EEF0A3EFF0ED30E013786506E684
:10A02F001870010690FCE3126CB7F97864803A90CF
:10A03F00FEE6E07002A3E0703C786CA6B5ED540E1E
:10A04F007864760008F618E6FE08E67807C333CE84
:10A05F0033CED8F9FF786CE6FDEE7864F6EF4D0855
:10A06F00F690FCE3126CB7F918E6FE08E6126D9451
:06A07F00F5B475B20122E8
:04004E0078680622A6
:0C87FA0041FC2A0141FC230041FC2B0043
:106F170090FD99E0FBA3E0FAA3E02404F9E43AFA30
:106F270012176654FD1217AC90FD99E0FBA3E0FA27
:106F3700A3E0F92290FC2FEFF090FC28E0FF7E0001
:106F470078307CFC7D017B017AFF798212174090B3
:106F5700FD9CE0FBA3E0FAA3E02403F9E43AFA027C
:106F6700176690FE0EE0FBA3E0FAA3E0229000155F
:106F770012177FFD2290FC27F0740FA3F0E490FC1A
:106F87002FF090FC28E0FF7E0078307CFC7D017BB1
:106F9700017AFF798222740B90FD33F0E4A3F0A30A
:106FA70004F0A374FCF0A3742FF02290001C021CC1
:106FB7002B900016021C2BEBF0A3EAF0A3E9F022BA
:106FC700900009121C2B02176690FC27F0A374028D
:106FD700F090FC2AE090FC2FF090FF82E090FC30CC
:106FE700F02290FD207401F0A374FCF0A37431F03B
:106FF7002290001FE4F5F002197A90000F121C2B63
:10700700EA494B22900009121C2B90000402177FBB
:10701700E490FC29F090FC272290001FE475F00112
:107027001218E1FEC3E5F022900019021C2B90FD17
:10703700ED7401F0A374FCF0A37424F02290FC27F4
:10704700F07401A3F090FC2AE090FC2F2290FD43FE
:107057007401F0A374FFF0A37480F0221217BE7BB3
:10706700007A00790022A37401F0A374FCF0A374E2
:10707700402290000202177F90FF82E0FF90FC30D1
:10708700F07E0078317CFC7D017B017AFF798322D9
:10709700F0A37401F0E490FC2FF090FECE22900054
:1070A7000102177F90FC27E090FD33F090FC28E069
:1070B70090FD34F0A374012290000302177F12178A
:1070C700AC90FE0E2290FC27F07401A3F090FF9283
:1070D700E02254FD1217AC90FECE22900001E4028C
:1070E70017BE12174090FECE2290001F1218A9C398
:1070F700942CE5F094012290000502177F90001F61
:10710700E475F03212197A740722121C2BE9240154
:1071170022121C2BE9240222900002E40217BEF07F
:1071270090FF82E0240390FC28F0229000151217AC
:0C7137007FFF7B0122121766D394012217
:10AB510090FE02126FBE90FE02E0F9A3E0FAA3E0BC
:10AB610090FC2CC9126FBF90FE05E0F9A3E0FAA397
:10AB7100E090FDC9C9126FBF90FE02126F320286CA
:01AB81002AA9
:1080ED0090FECB126FBE90FECB126F32E41217AC26
:1080FD0090FECB126F321270E212711F900003E4EA
:10810D001217BE90000474401217BE900005E412C1
:10811D007063C003C002C00190FECB126F3290009D
:10812D0006121C5B127066C003C002C00190FECB2C
:10813D00126F32900009121C5B127066C003C002F0
:10814D00C00190FECB126F3290000C121C5B1270AE
:10815D0066C003C002C00190FECB126F3290000FBB
:10816D00121C5B127066C003C002C00190FECB12E0
:10817D006F32900012121C5B90FECB126F3290008A
:10818D0015ED127063C003C002C00190FECB126FDB
:10819D0032900016121C5B127066C003C002C00143
:1081AD0090FECB126F32900019121C5B127066C0DC
:1081BD0003C002C00190FECB126F3290001C121C46
:1081CD005B90FECB126F3290001FE4F5F002197A2E
:06B3A30090FC23EFF022F4
:1093DC0090FCFA126FBE90FD00126F32C003C002F7
:1093EC00C00190FCFD126F32900009121C5B90FDC5
:1093FC0003126F32C003C002C00190FCFD126F3229
:10940C0090000C121C5B90FCFD126F32C003C0026A
:10941C00C00190FD03126F32900006121C5BC0035A
:10942C00C002C00190FD00126F32900006121C5B4E
:10943C0090FCFA126F32C003C002C00190FD0312FF
:10944C006F32900016121C5BC003C002C00190FD6D
:10945C0000126F32900016121C5BC003C002C001D8
:0D946C0090FCFD126F32900019121C5B2263
:1097E90090FD06126FBE90FD0C126F32C003C002CD
:1097F900C00190FD09126F3290000F121C5B90FDA1
:109809000F126F32C003C002C00190FD09126F32FE
:10981900900012121C5B90FD09126F32C003C00246
:10982900C00190FD0F126F32900006121C5BC0033D
:10983900C002C00190FD0C126F32900006121C5B31
:1098490090FD06126F32C003C002C00190FD0F12D5
:109859006F32900016121C5BC003C002C00190FD5C
:0B9869000C126F32900016121C5B22E4
:10B26D00C003C002C00190FE0B126F3290001C1281
:03B27D001C5B2235
:103AFE0090FECE126FBE90FECE126F3212987450A0
:103B0E002590FC2C126F32124089126F3212702FD8
:103B1E00124093126F6C2404126F621270D9126FDE
:103B2E003274011217AC90FECE126F321270A530A5
:103B3E00E61E1270E27D40128AF990FECE126F6C74
:103B4E002404126F621270D9126F3274011217AC04
:103B5E0090FECE126F3212176614604D14607B14F5
:103B6E007003023C1F24FE7003023C5524056003C3
:103B7E00023D0A90FC2C126F32124089126F3212E3
:103B8E00702F124093126F32126FB2E4FD1281DD6C
:103B9E0090FECE126F32126FB27D0112A25D90FEB8
:103BAE00CE126F327401023D0790FECE126F3212AA
:103BBE0098FC4003023D0A90FECE126F32126FF84F
:103BCE0012B25A90FECE126F3212702F12ABDB90E1
:103BDE00FECE126F327402023D0790FECE126F328D
:103BEE00128F67502A90FECE126F321270209419E7
:103BFE00EE94005003023D0A126FF812702F129BC2
:103C0E009D1201EE90FECE126F327403023D0780BC
:103C1E002A90FECE126F3212702F12AB1FEF601B66
:103C2E0090FECE126F321270209432EE940050033A
:103C3E00023D0A126FF87405023D0790FECE126F18
:103C4E0032126FF8023D0A90FECE126F3212702FB2
:103C5E0012B2FFEF601490FECE126F3212702F125E
:103C6E00B199EF90FECE6020801290FECE126F3290
:103C7E0012702F12B199EF90FECE600C126F6C2461
:103C8E0004126F624402800A126F6C2404126F6277
:103C9E0054FD1217AC90FECE126F321270F0500A15
:103CAE0090001FE475F00112192D12702F12AB1F28
:103CBE00EF704990FECE126F321270F0402E1270DD
:103CCE001130E11312ABAF90FECE126F6C240412C2
:103CDE006F6254FD1217AC90FECE126F327D8012C1
:103CEE008AF990FECE126F327402800D90FECE12C3
:103CFE006F6C2404126F6254FD1217AC90FECE123C
:103D0E006F32126FB2129A924003023F4F90FECE64
:103D1E00126F32126FB2127054A3E4F0A37413F048
:103D2E0012A75290FF80E0B410004003023F4F9064
:103D3E003D44F8282873023D74023D95023D9C02D5
:103D4E003DA3023DAE023DBE023DD2023DF7023E14
:103D5E000D023E22023E32023E47023E60023E7697
:103D6E00023E86023EA51270170412712690FF9233
:103D7E00E0B40F0890FC2F740FF08005E490FC2F38
:103D8E00F012707F023E02127017741980171270B3
:103D9E0017741A801090FECE126F327D04023F4CC3
:103DAE00127017741C127097126F327D40023F4CC6
:103DBE001270177406F0E4A3F090FECE126F327DEF
:103DCE0040023F4C78247CFC126F947E007F0312DD
:103DDE0070E9126F32126FB212703512AA8290FE13
:103DEE00CE126F327D10023F4C1270177410F0A37A
:103DFE0014126F831270E9126F327D40023F4CE451
:103E0E0090FC29F07412126F7C1270E9126F327DE1
:103E1E0040023F4C1270177413127097126F327D5E
:103E2E0040023F4CE490FC29F0741D126F7C12701E
:103E3E00E9126F327D40023F4C127017741EF0A3D0
:103E4E007402F0E4126FDC90FECE126F327D4002EF
:103E5E003F4C1270177415F07406126F821270E9CF
:103E6E00126F327D40023F4C12701774161270970B
:103E7E00126F327D40023F4C90FC297401F090FC91
:103E8E0027741FF0A37402F0E4126FDC90FECE12C2
:103E9E006F327D40023F4C90FF81126FDB90FC2F02
:103EAE00E064057047A3E0702390FECE126F3212CD
:103EBE006FB290FDF3126FEC12A0E8EF6003023FB9
:103ECE004F90FECE126F327D80023F4C90FECE128E
:103EDE006F32126FB290FDF3126FEC12A0E8EF602A
:103EEE006090FECE126F327D80023F4C90FC30E02F
:103EFE00702190FECE126F32126FB290FD29126FAA
:103F0E00EC12706D12409A703890FECE126F327DA8
:103F1E0080802B90FECE126F32126FB290FD29125E
:103F2E006FEC12706D12409A601790FC2FE0FF90AC
:103F3E00FC2AE0B5070B90FECE126F327D801299EF
:103F4E008490FECE126F32127079FD600C1299843D
:103F5E0090FECE126F3212711F90FECE126F321281
:103F6E0070BF30E328E9126F6054F71270DB126FE6
:103F7E0032126FB2C0037406126F9FD003E4FD12AB
:103F8E009EE890FECE126F327D0802998490FECE8E
:103F9E00126F321270BF30E42EE9126F6054EF12BE
:103FAE0070DB126F32126FB212703512AA8290FE4F
:103FBE00CE126F32126FB2C00390FD33740CF0E468
:103FCE00A3F0A30402407E90FECE126F321270BF99
:103FDE0030E63CE9126F6054BF1217AC90FC27E03C
:103FEE00B4071A90FECE126F32126FB290FDFF74AC
:103FFE0001F0A374FCF0A37430F012AAB790FECEB9
:10400E00126F32126FB21270AB126FA80240839011
:10401E00FECE126F321270BF30E517E9126F605488
:10402E00DF1270DB126F32126FB290FC2AE0FD02CB
:10403E009D1690FECE126F321270BF30E73CE91221
:10404E006F60547F1217AC1270177418F0A37402BD
:10405E00F090FC2F14F0E4A3F090FECE126F32120B
:10406E006FB2C00390FD337418F0A37402F0A31462
:10407E00126FA8D003E4FD129EE822129A0C12B21F
:10408E005A90FECE2212ABDB90FECE22F0128A3078
:06409E0090FC2AEFF02265
:1055470090FE0E126FBE900006121C2B90FE1112D9
:105557006FBE90FE0E126F32129874400E90FE0EC0
:10556700126F321270A5700302564390FE0E126F2F
:1055770032126FB8C003C002C00190FE0E126F3224
:10558700126F74D001D002D00312B037126F6924A2
:1055970004126F6254FD1270C5126F32126FB8C0D9
:1055A70003C002C00190FE0E126F32126F74D00159
:1055B700D002D00312AF7290FE0E126F32126FB884
:1055C700C003C002C00190FE0E126F32126F74D07A
:1055D70001D002D00312593E126F3212702F12AB54
:1055E700DB90FE0E126F32126FF81270A530E70AC9
:1055F70090FE0E126F327D80802190FE0E126F3268
:105607001270A530E62290FE11126F6C2401126F02
:105617006244401270C5126F327D40128AF990FEC3
:105627000E126F327402800890FE0E126F327401F0
:105637001217AC90FE0E126F321270E290FE0E122D
:105647006F321217661470030257F9147003025869
:105657001214700302582B14700302589E1470031F
:105667000258A8240560030258DB126FB8C003C0B4
:1056770002C00190FE0E126F32126F74D001D00279
:10568700D00312593E126F3212702F12ABDB90FE0D
:1056970011126F3212176670411270FE90FE0E30B3
:1056A700E40C126F6C2405126F624410800A126FAB
:1056B7006C2405126F6254EF1217AC90FE11126F33
:1056C700321270FE90FE0E30E5030257A7126F6C80
:1056D7002405126F6254DF0257B1126F6924051255
:1056E7006F6254EF1217AC54DF1270C5126F32128B
:1056F7006FB8C003C002C00190FE0E126F32126F66
:1057070074D001D002D00312AF3090FE0E126F3268
:1057170012702F129B9D90FE0E126F32126FB8C03F
:1057270003C002C00190FE0E126F32126F74D001D7
:10573700D002D00312A80DEF700D126F6924051265
:105747006F6244100257B190FE0E126F32126FB89B
:10575700C003C002C00190FE0E126F32126F749028
:10576700FD7A127057D001D002D0031290BAEF70B1
:105777000C126F692405126F624410802D126F6935
:105787002405126F6254EF1217AC90FE0E126F329F
:105797001271327AFF7980128D48EF701090FE0EE9
:1057A700126F6C2405126F6244200217AC126F69E6
:1057B7002405126F6254DF1217AC90FE0E126F327F
:1057C700126FB8C003C002C00190FE0E126F3212F2
:1057D7006F74D001D002D00312B01790FE0E126F73
:1057E7003212702F12ABDB90FE0E126F3274010271
:1057F70058D690FE0E126F321298FC40030258E4FE
:1058070090FE0E126F3274020258D690FE0E126F7F
:1058170032128F6740030258E490FE0E126F327403
:10582700030258D690FE11126F32121766D39403F3
:1058370050030258E490FE0E126F32126FB8C00385
:10584700C002C00190FE0E126F32126F74D001D0E9
:1058570002D00312AF3090FE0E126F3212702F1269
:105867009B9D90FE0E126F32126FB8C003C002C02C
:105877000190FE0E126F32126F74D001D002D00366
:1058870012AFB4126F692404126F6244011270C51B
:10589700126F327404803890FE0E126F32740580D6
:1058A7002E90FE11126F3212701190FE0E30E1151C
:1058B700126F6C2404126F6244021270C5126F32A9
:1058C700127104800A126F6C2404126F6254FD1265
:1058D70017AC800990FE0E126F321245F790FE0E3C
:1058E700126F32129C9A126F6950092404126F6268
:1058F700441080072404126F6254EF1217AC90FE15
:105907000E126F32127079FD600C12998490FE0EA0
:10591700126F3212711F90FE0E126F321270BFFF9C
:10592700601490FE11126F594F1270C5126F3290AA
:0E5937000003E41217BE2212B01790FE0E22DB
:1021860090FD99126FBE900006121C2B90FD9C12BA
:102196006FBE126F2F12713C500302226F126FB87E
:1021A600C003C002C001126F2F126F74D001D0029B
:1021B600D003129E7EEF6011126F2F12701120E570
:1021C600081270A5700302226F126F2F126FB8C02B
:1021D60003C002C001126F2F126F74D001D002D05B
:1021E6000312B037126F17126FB8C003C002C001D6
:1021F600126F2F126F74D001D002D00312AF721279
:102206006F2F126FB8C003C002C001126F2F126F7A
:1022160074D001D002D00312B017126F2F126FF8CC
:102226001270A530E72B126F2F126FB8C003C002D1
:10223600C001126F2F126F74D001D002D003129E0C
:102246007EEF90FD996005126F32800E126F32801C
:102256000D126F2F1270A530E6047402800274010D
:102266001217AC126F2F1270E2126F2F121766B48C
:1022760007004003022673902284F828287302225E
:10228600990223D102250A0225220225940225A5B8
:10229600022601126FB8C003C002C001126F2F12CE
:1022A6006F74D001D002D00312B01790FD9C126F4C
:1022B60032121766704B1270FE90FD9930E40C12C4
:1022C6006F6C2405126F624410800A126F6C24052D
:1022D600126F6254EF1217AC90FD9C126F3212709F
:1022E600FE90FD9930E50D126F6C2405126F624465
:1022F60020022392126F6C2405126F6254DF0223B0
:102306009290FD99126F6C2405126F6254EF1217AA
:10231600AC54DF126F2C126FB8C003C002C001129A
:102326006F2F126F74D001D002D00312AF30126F2C
:102336002F126FB8C003C002C001126F2F126F7444
:10234600D001D002D00312A80DEF700F90FD9912A4
:102356006F6C2405126F6244108031126F2F126F5A
:10236600B8C003C002C001126F2F126F7490FD7ABD
:10237600127057D001D002D0031290BAEF701090AD
:10238600FD99126F6C2405126F6244100217AC900F
:10239600FD99126F6C2405126F6254EF1217AC127E
:1023A6006F2F126FB8C003C002C001126F2F126FD9
:1023B60074D001D002D00312B017126F2F126FB271
:1023C6007D041281DD126F2F022708126F2F126F04
:1023D600B8C003C002C001126F2F126F74D001D0B3
:1023E60002D003129E7E90FD9FEFF0700302271528
:1023F600126F2F12701130E5030227151270209408
:102406000AEE940050030227151271327AFA799671
:10241600127143EF601F126F2F90001F1218A9C38D
:102426009419E5F094005003022715E92405126F6C
:10243600624440800D90FD99126F6C2405126F6204
:1024460054BF1217AC126F2F126FF87B017AFA790C
:10245600961296D1EF90FD99604E126F6C2404127D
:102466006F6244011217AC7B017AFA7996129FB912
:10247600749A2FF974FA3EFA90FDE77401126FBF51
:10248600126F2F126FB212AA4D126F2F126FB27DFA
:102496000212A25D126F2F126FB2C003126F9DD08F
:1024A60003E4FD129EE8800D126F6C2404126F6225
:1024B60054FE1217AC126F2F126FB812B2FFEF60F4
:1024C6000D126F2F12701130E6047F0180027F001B
:1024D60090FC7CEFF090FC797401F0A374FAF0A301
:1024E6007496F090FC2C126F32120280EF601090FE
:1024F600FD9C126F6C2401126F6244401217AC12DD
:102506006F2F8013126F2F127020940AEE940050D2
:1025160003022715126FF8740302270A90FD9C1216
:102526006F32121766D394035003022715126F2FCA
:10253600126FB8C003C002C001126F2F126F74D0A1
:1025460001D002D00312AF30126F2F12701130E09B
:102556001A126FB8C003C002C001126F2F126F7437
:10256600D001D002D00312AFB4801B126F2F126FAE
:10257600B8C003C002C001126F2F126F74D001D011
:1025860002D00312B057126F2F740402270A126F7B
:102596002F126FB812A8FF126F2F740502270A12A6
:1025A6006F2F126FB8C003C002C001126F2F126FD7
:1025B60074D001D002D003120026EF7026126F2FBE
:1025C600126FB8C003C002C001126F2F126F74D011
:1025D60001D002D00312B017126F2F126FF87406D3
:1025E60002270A90FD9C126F3212701120E103023D
:1025F6002715126F2F12710402270A126F2F1270FD
:102606002094FAEE94005003022715126FF8126F09
:10261600B8C003C002C001126F2F126F74D001D070
:1026260002D00312AF3012AE9D126F2F126FB8C0D8
:1026360003C002C001126F2F126F74D001D002D0F6
:1026460003120026EF6008126F2F74031217AC12E4
:102656006F2F126FB8C003C002C001126F2F126F26
:1026660074D001D002D00312B017022715126F2FB3
:10267600126FB8C003C002C001126F2F126F74D060
:1026860001D002D003120026EF6020126F2F126FC6
:10269600B8C003C002C001126F2F126F74D001D0F0
:1026A60002D003129E7EEF6401605E126F2F126FDE
:1026B600B8C003C002C001126F2F126F74D001D0D0
:1026C60002D00312B037126F17126FB8C003C002E0
:1026D600C001126F2F126F74D001D002D00312AF57
:1026E60072126F2F126FB8C003C002C001126F2F93
:1026F600126F74D001D002D00312B017126F2F12CE
:102706006FF874011217AC8006126F2F1245F7127C
:102716006F2F121766FF640C6019EFD394024013F3
:10272600EF6406600E90FA90E020E70790FA8FE0DB
:1027360030E30AE92404126F624410800D90FD997B
:10274600126F6C2404126F6254EF1217AC126F2FC3
:10275600126FB2129A9240030229AC126F2F126FB7
:10276600B2127054A3E4F0A37413F012A75290FFB0
:1027760080E0121CB427BB0027FB03280605280EA1
:102786000628300728580828770928950C28B70DF9
:1027960028E61028EE11290312291113292C1429D1
:1027A6001115293D16294A17295718296A19297911
:1027B6001A000029AC90FF92E0FDB405047E01806A
:1027C600027E0090FC29EEF090FC2774011271261F
:1027D600EDB4050890FC2F7405F0801390FF92E08D
:1027E600B40F0890FC2F740FF0800412704CF01296
:1027F600707F02285090FC27741BF0E4A302288CFB
:10280600126F5644080229A978247CFC126F947E24
:10281600007F03121740126F2F126FB2127035121B
:10282600AA82126F5644100229A990FC277410F050
:10283600A314F090FF92E0B405047F05800590FC98
:102846002AE0FF90FC2FEF126F88126F534440026C
:1028560029A990FC277412F0740F1270D2B40504E3
:102866007F05800590FC2AE0FF126F3B4440022959
:10287600A974131270CCB405047F05800590FC2A58
:10288600E0FF90FC2FEFF0126F5644400229A9900A
:10289600FC277415F0A37406F090FF92E0B40504CB
:1028A6007F05800590FC2AE0FF126F3B4440022919
:1028B600A974161270CCFFB405047E05800590FC41
:1028C6002AE0FE90FC2FEEF0126F5644401217AC31
:1028D600EF640560030229AC126F5644800229A9F1
:1028E600126F5644200229A97407127044F0126F21
:1028F600907E007F08126F5344400229A974081283
:102906007044F0126F5644400229A990FC277409BE
:10291600F0741112704AF0126F907E007F10126FE1
:102926005344400229A978407CFC126F947E007FB4
:102936000E1217400229AC7414126FD0126F56444F
:10294600400229A9740D126FD0126F564440022915
:10295600A990FC27740EF0A3740912704B126F3FF6
:102966004440803F90FC27740F126FD3126F564479
:1029760040803090FC277417F0A37403F090FC2F6E
:102986007405126FDF90FF84E0600790FC2AE0FF79
:1029960080027F0090FC31EFF0126F564440121710
:1029A600AC44801217AC126F2F12707930E127E910
:1029B6002402126F6254FD1217ACE490FC2FF01241
:1029C6006F2F126FB290FD33741AF0A37401F0A347
:1029D600126FA8022B10126F2F12707930E21DE9C8
:1029E6002402126F6254FB126F2C126FB2C0039056
:1029F600FD33741B126FA2D003022B10126F2F121D
:102A0600707930E31DE92402126F6254F7126F2CBD
:102A1600126FB2C00390FD337406126FA2D0030288
:102A26002B10126F2F12707930E429E92402126FED
:102A36006254EF126F2C126FB212703512AA821204
:102A46006F2F126FB2C00390FD33740C126FA2D0B9
:102A560003022B10126F2F12707930E61CE9240244
:102A6600126F6254BF126F2C126FB290FC29E0FDF8
:102A76001270AB126FA8022B43126F2F12707920BF
:102A8600E703022B56E92402126F62547F1217AC39
:102A960090FC2FE064057042A3E064047015126F89
:102AA6002F126FB2126FE9A3E4F0A3F0A3F0127D28
:102AB600A1800A90FC30E0700FA374FFF0126F2F14
:102AC600126FB27D0202A25D126F2F126FB2126FE9
:102AD600E9A3E4F0A3F0A3022B5290FC30E06404D7
:102AE600702C126F2F126FB2126FE912706DF01206
:102AF6007DA1126F2F126FB27D0212A25D126F2F8F
:102B0600126FB2C003126F9DD003E4FD802F90FCBC
:102B160030E0702CA37404F0126F2F126FB27D0494
:102B26001281DD126F2F126FB27D0212A25D126F3B
:102B36002F126FB2C003126F9DD003E4FD029EE810
:102B4600126F2F126FB2126FE912706DF0127DA123
:012B5600225C
:0BB35500E92404126F6244200217ACD0
:0BB36000E92404126F6254DF0217ACF6
:1098740090FED1126FBE90FED1126F321270016051
:109884005290FED1126F3290001212700460449014
:10989400FED1126F3212713C4037126FC7640170EF
:1098A4003090FED1126F3290000C126FCA640170B6
:1098B4002090FED1126F3290000F126FCAB40111C2
:1098C40090FED1126F32900012126FCAB40102D30B
:1098D40022C32290FED1126F3212713C4018126FD3
:1098E400C7B4011290FED1126F3290000C126FCAED
:0898F400B40103D38001C3227B
:1098FC0090FED4126FBE90FED4126F3212700160C3
:10990C005390FED4126F3290001212700460459086
:10991C00FED4126F32126FC7D39401503390FED421
:10992C00126F3290000C126FCAD39401502290FE29
:10993C00D4126F3290000F126FCAD3940150119051
:10994C00FED4126F32900012126FCAD394014002EF
:10995C00D322C32290FED4126F32126FC7D394015C
:10996C00501190FED4126F3290000C126FCAD39427
:08997C00014003D38001C32266
:108F670090FED7126FBE90FED7126F32127001605B
:108F77006B90FED7126F32900012127004605D90F2
:108F8700FED7126F32126FC7FF64036006EFD394E8
:108F970001504790FED7126F3290000C126FCAFF34
:108FA70064036006EFD39401503090FED7126F32FE
:108FB70090000F126FCAFF64036006EFD39401504D
:108FC7001990FED7126F32900012126FCAFF640316
:108FD7006006EFD394015002D322C32290FED7122A
:108FE7006F32126FC7FF64036006EFD39401501A04
:108FF70090FED7126F3290000C126FCAFF640360A5
:0C90070006EFD394015003D38001C32274
:109C9A0090FEDA126FBE90FEDA126F321270016015
:109CAA004B90FEDA126F32900012127004603D90EF
:109CBA00FEDA126F3212700B30E42F90FEDA126F56
:109CCA003290000C12700E30E42090FEDA126F32DD
:109CDA0090000F12700E30E41190FEDA126F32907B
:109CEA00001212700E30E402D322C32290FEDA125E
:109CFA006F3212700B30E41290FEDA126F3290005B
:0C9D0A000C12700E30E403D38001C32261
:108AF90090FEDD126FBE90FEDD126F3290000912FA
:108B09007004602190FEDD126F32126FC7D3940397
:108B1900401390FEDD126F32900009127111126F2D
:108B2900624D1217AC90FEDD126F3290000C12707C
:108B390004602490FEDD126F3290000C126FCAD3CC
:108B49009403401390FEDD126F3290000C127111E4
:108B5900126F624D1217AC90FEDD126F3212700166
:108B6900602490FEDD126F3290000F126FCAD39409
:108B790003401390FEDD126F3290000F1271111233
:108B89006F624D1217AC90FEDD126F329000121217
:108B99007004602490FEDD126F32900012126FCAC9
:108BA900D39403401390FEDD126F329000121271BC
:098BB90011126F624D1217AC227B
:1099840090FEE0126FBE90FEE0126F32900009125A
:109994007004601390FEE0126F3290000912711887
:1099A400126F624D1217AC90FEE0126F3290000CF1
:1099B400127004601390FEE0126F3290000C12716A
:1099C40018126F624D1217AC90FEE0126F321270D3
:1099D40001601390FEE0126F3290000F12711812A2
:1099E4006F624D1217AC90FEE0126F3290001212AB
:1099F4007004601390FEE0126F329000121271181E
:089A0400126F624D1217AC2233
:10880600182F00000000000000000000000000001B
:0A8816000000000000000000000058
:10A3060085128385138222860308E6FA08E64A4BFD
:10A316002208E6FA08E6F9021CDAA3E0FEA3E0FF4B
:10A326002290FFFF121CE0EFF0C2A922AA06AB079B
:10A3360090FEF6E025E0227C001217F2EF22F8A646
:10A346000308A60208A60122F8E6FE08E6FFE4FCDA
:02A35600FD22E6
:1076AA0090FFFF121CE0EBF090FFFE121CE0ECF0E2
:1076BA00A3EDF012A327E58954FCFE12A306E0FB12
:1076CA004EF589900003121D04E044C0F58B90FE2C
:1076DA00FAE014605A1470030277812402600302EC
:1076EA0077D312A30612A320EE54FE7009758C16E6
:1076FA00EEC313EF805F12A30612A320EE54FC70B0
:10770A0010758C2DEF7802CEC313CE13D8F90277F9
:10771A00C212A30612A320D394EAEE9415500B7555
:10772A008CFC7D1612A33D0277C2AF030277CC12FE
:10773A00A306A3E0FEEE700C758C0E12A306A3A39B
:10774A00E00277C2EE54FE700F758C1D12A306A3D9
:10775A00E0C313A3E013806012A30612A320D394FC
:10776A00EFEE9410500A758CFE7D1112A33D8048ED
:10777A0012A306E0FF804B12A306A3E0FEEE700BF5
:10778A00758C1012A306A3A3E0802DEE54FE700F91
:10779A00758C2112A306A3E0C313A3E01380191268
:1077AA00A30612A320D394EFEE94105010758CFE0A
:1077BA007C007D0F1217F2EF14F58D800C12A306D0
:1077CA00E0FF12B0967F00803CAF8C12A306E0FD6A
:1077DA0025E02427F8760008A607AF8DED25E024DA
:1077EA0047F8760008A6077401A805088002C33383
:1077FA00D8FCF5887410A805088002C333D8FC4267
:0B780A0089D2A97F01900004021CE05D
:10B0960012A32712A306E0FF7410A807088002C3B4
:0EB0A60033D8FCF45289D2A9900001021CE0BC
:0BB36B00EF75F003A4242F12A344226E
:0BB37600EF75F003A4243B12A3442257
:108BC20090FEF6EFF0FBC2A9E58954FC4BF589AFA4
:108BD2008C7862760008A607AF8DE4FCFDFE785E15
:108BE200121BE2EB25E0244712A34E785E121BA56E
:108BF200C3EF9BFFEE9AFEED99FDEC98FCC004A931
:108C02000512A332242712A34ED0001219A7C004C2
:108C1200C00512A3322428F9C3E7786396FF19E747
:108C22001896FEE4FCFDD001D000EB2FFFEA3EFED9
:108C3200ED39FDEC38FC785E121BE290FEFAE0148E
:108C4200601C14602424027033E47F19FEFDFC785A
:108C52005E121BA51219A7E47B207A018014785EAC
:108C6200121B99E47B0FFA8009785E121B99E47B50
:108C720011FAF9F8121A32785E121BE2D2A9786060
:068C8200E6FE08E6FF22F9
:03000B000283AAC3
:1083AA00C0E0C0F0C083C082C0D075D000C000C099
:1083BA0001C002C003C004C005C006C0073088124D
:1083CA00782F12A30D6005782F12A3177588010262
:1083DA008468308912783212A30D6005783212A3AC
:1083EA0017758802028468308A12783512A30D60E4
:1083FA0005783512A317758804028468308B1178C2
:10840A003812A30D6005783812A317758808804EB4
:10841A00308C11783B12A30D6005783B12A31775B7
:10842A008810803A308D11783E12A30D6005783E8F
:10843A0012A3177588208026308E11784112A30D59
:10844A006005784112A3177588408012308F0F7823
:10845A004412A30D6005784412A317758880D007CB
:10846A00D006D005D004D003D002D001D000D0D09D
:09847A00D082D083D0F0D0E032B2
:08B38B00E5FF54077869F62282
:0500060012B38B002283
:10B0B40012B38BE6FF700476098008EFB4010C78B4
:0CB0C4006976027869E660031680F822C5
:10AF0D0012B38BE6FF7004760C800FEFB401067858
:10AF1D006976048005EFB40209227869E6600316AC
:03AF2D0080F82287
:10AE9D0012B38BE6FF700476178012EFB4010678BB
:10AEAD006976098008EFB4020C786976027869E654
:06AEBD0060031680F8227C
:10A4460090FEFAE014601314602624027036E5FFCD
:10A45600540770387869760D802AE5FF5407146032
:10A466000904702878697615801A7869760380144D
:10A47600E5FF54071460090470127869761A80049F
:0DA48600786976057869E660031680F82293
:109C1C0090FEFAE014602714604424027067E5FF9C
:109C2C00540714600D146010240270617869764535
:109C3C0080537869761B804D786976058047E5FFFF
:109C4C00540714600D146010240270417869765F1B
:109C5C00803378697628802D7869760C8027E5FF2B
:109C6C0054071460101460131460162403701E78CB
:109C7C0069766D80107869762F800A7869760F8006
:0E9C8C0004E47869F67869E660031680F82231
:10951200303204D2AED2BE90FEFAE0146030146053
:109522005624027079E5FF54071460101460131476
:109532006016240370707869767E80627869763767
:10954200805C786976138056786976018050E5FFF1
:1095520054071460101460131460162403704778C3
:109562006976A980397869764C80337869761E806D
:109572002D786976078027E5FF5407146010146080
:10958200131460162403701E786976C080107869FF
:109592007658800A7869762480047869760A786930
:0795A200E660031680F822C9
:107AE300303204D2AED2BE90FEFAE0146078147045
:107AF30003027BD324026003027C32E5FF5407B404
:107B030007004003027C42907B11F8282873027B14
:107B130026027B2D027B37027B41027B4B027B5586
:107B2300027B5F786A7603027BC5786A7601087602
:107B330084027C32786A76000876BC027C32786AEA
:107B43007600087658027C32786A76000876260238
:107B53007C32786A760008760D027C32786A760089
:107B6300087601027C32E5FF5407B40700400302A4
:107B73007C42907B7CF8282873027B91027B9B02DA
:107B83007BA5027BAF027BB8027BC1027BCA786A0A
:107B93007604087607027C32786A76010876FD025D
:107BA3007C32786A76000876F9027C32786A76004D
:107BB300087676807A786A76000876358071786AF6
:107BC30076000876158068786A7600087604805F08
:107BD300E5FF5407B407005066907BE3F828287349
:107BE300027BF8027C01027C0A027C10027C1902EF
:107BF3007C22027C2B786A76040876898031786A45
:107C0300760208763E8028786A76018016786A764E
:107C1300000876878019786A760008763D801078A8
:107C23006A76000876198007786A760008760678FF
:107C33006BE61846600908E6161870F31680F02202
:10B2B5007869760A7869E6166005127AE380F522E0
:10B2C500786976647869E6166005127AE380F52276
:0CB31900AE071FEE600512951280F522B1
:0CB32500AE071FEE6005127AE380F522EF
:0CB33100AE071FEE600512B2B580F522D9
:0CB33D00AE071FEE600512B2C580F522BD
:108820000F4F0000000000000000000000000000EA
:018830000047
:10AD340090FFFF121CE0EFF08512838513822286B8
:10AD44000308E6FA08E64A4B2208E6FA08E6F9029E
:0AAD54001CDAE0FF7401A8070822D2
:10A7910090FFFF121CE0EDF012AD3412AD568002B5
:10A7A100C333D8FC12AD3CF0E0FF42F312AD3CA341
:10A7B100E06005EF42F4800712AD3CE0F452F41280
:0FA7C100AD3CE0F5F6D2A842F5900002021CE094
:10B1070012AD3412AD568002C333D8FC12AD3CF0F9
:0AB11700E055F2FF900001021CE079
:10B1F40012AD3412AD568002C333D8FCF452F5902C
:05B204000001021CE046
:10B29300EF75F003A4244FF8A60308A60208A6013D
:01B2A3002288
:0300030002920066
:10920000C0E0C0F0C083C082C0D075D000C000C034
:1092100001C002C003C004C005C006C007E5F55583
:10922000F6F523301811784F12AD436005784F12D0
:10923000AD4D75F601804E301911785212AD436074
:1092400005785212AD4D75F602803A301A117855F4
:1092500012AD436005785512AD4D75F60480263089
:109260001B11785812AD436005785812AD4D75F654
:10927000088012301C0F785B12AD436005785B12DA
:10928000AD4D75F610D007D006D005D004D003D070
:1092900002D001D000D0D0D082D083D0F0D0E03244
:1088310046FD50000000000000061400000000008A
:018841000036
:1096400075BC01C390FCF8E094A890FCF7E094612D
:1096500022781408E6FA08E6F5828A83021CDE788E
:1096600014860308E6FA08E64A4B2290FCF2E0FE74
:10967000A3E0FF90FCF5E0FCA3E0FDC39FEC9E227D
:10968000F5B7E490FCF7F0A3F022E5BC540690FC9B
:10969000F9F022ED5401C4333354C022781C08067B
:1096A000E6188606222456F582E434FDF5832290DE
:1096B000FCF7E004F02290FCF97403F022E490FC43
:1096C000F5F0A3F02290FCEFE0FBA3E0FAA3E0F9B1
:0196D0002277
:10AA1700EF6019D2BAED6006D2B6D2B78004D2B4CD
:10AA2700D2B543BB04E490FD57F08017D2B9ED606F
:10AA370006D2B2D2B38004D2B0D2B143BB02E49003
:06AA4700FD56F002ACB563
:10ACB500EF600543BB01800353BBFEEDB4020CEB13
:10ACC5005403C454F0FF129693800C12969344805B
:0BACD500FFEB5403C454F04FF5B7220E
:10A8870090FE63EBF0EF6014D2BAED6006D2B6D259
:10A89700B78004D2B4D2B543BB048012D2B9ED60FD
:10A8A70006D2B2D2B38004D2B0D2B143BB0212AE49
:0CA8B700E990FE63E0F5B3A3E0F5B622E3
:10AEE900E5BB54FE4FF5BBEDB40208129694442E0F
:10AEF900F5B12212969344AEF5B175B4FF75B21F40
:04AF090043B101222D
:10B1B000EF75F003A42450F582E434FDF583EBF041
:07B1C000A3EAF0A3E9F0226D
:10B2A400EF75F003A42414F8A60308A60208A60167
:01B2B4002277
:1074FF0090FCEDEFF0A3EDF0A3EBF0A3EAF0A3E91E
:10750F00F01296BDA3F0A3F0A3F090FCEDE0FE12F5
:10751F0096A5E060037F012274562E1296A7740180
:10752F00F0E5BB54FE4EF5BB75BC0190FCF4E020BA
:10753F00E12E90FCEEE0F5BDE5B754F14402129652
:10754F0080E5BC20E00D12769670031296AF12966E
:10755F004340EE129640500512968A80031296B65B
:10756F0090FCF9E0600302768790FCEEE020E003E8
:10757F000276051296BD12966B400302765890FC68
:10758F00F9E06003027658EF24FFFFEE34FFFEEDC3
:10759F00B50715ECB5061190FCF4E020E00AE5B74D
:1075AF0054F1440AF5B78008E5B754F14406F5B72E
:1075BF00129682E5BC20E00D12769670031296AFFC
:1075CF0012964340EE1296C590FCF5E0FEA3E0F54F
:1075DF00828E83E5BF1217BE129640500512968A0F
:1075EF0080031296B690FCF6E004F0700690FCF55E
:1075FF00E004F00275851296BD12966B504B90FC0D
:10760F00F9E070451296C58D828C8312177FF5BEF7
:10761F00E5B754F14406129680E5BC20E00D1276D2
:10762F00A070031296AF12964340EE12964050058B
:10763F0012968A80031296B690FCF6E004F070065C
:10764F0090FCF5E004F002760890FCF4E020E028CE
:10765F00E5B754F1440E129680E5BC20E00D12768A
:10766F00A070031296AF12964340EE12964050054B
:10767F0012968A80031296B690FCEDE01296A5E45E
:10768F00F090FCF9E0FF2212000690FCF8E004F005
:0B769F002212000690FCF8E004F0222C
:03004B00028EB86A
:108EB800C0E0C0F0C083C082C0D075D000C000C080
:108EC80001C002C003C004C005C006C00790FEF779
:108ED800E5BBF053BBFEE5B230E11912965F600FB7
:108EE80012969C70010614FF781AE6FD12965175C9
:108EF800B202804AE5B230E211781AE620E0064470
:108F080001F675B20175B2048034E5B230E3107829
:108F18001C7600087600781AA6B575B208801FE599
:108F2800B230E01A781AE6FD30E01312965F600B53
:108F380012969C70010614FF12965175B20190FEAC
:108F4800F7E0F5BBD007D006D005D004D003D00297
:0F8F5800D001D000D0D0D082D083D0F0D0E03282
:03005300028C8894
:108C8800C0E0C0F0C083C082C0D075D000C000C0B2
:108C980001C002C003C004C005C006C00790FEF8AA
:108CA800E5BBF0E5BB54FE4401F5BBE5B230E11F7E
:108CB80078171296616013781E12969E700106143A
:108CC800FF781BE6FD781712965375B2028050E5BF
:108CD800B230E211781BE620E0064401F675B201D5
:108CE80075B204803AE5B230E310781E7600087653
:108CF80000781BA6B575B2088025E5B230E020786B
:108D08001BE6FD30E0197817129661600F781E1285
:108D1800969E70010614FF781712965375B201904B
:108D2800FEF8E0F5BBD007D006D005D004D003D0BC
:108D380002D001D000D0D0D082D083D0F0D0E032A1
:10ADB100EBF0A3EAF0A3E9F02290FE34E0FBA3E07C
:10ADC100FAA3E0F92275A102439A03439C03539B22
:09ADD100FC227B017AFF7980224B
:10915F0090FE25EEF0A3EFF0A3EDF090FEFAE014F1
:10916F00600F146014240270507F007ED07D028047
:10917F000E7F807EA97D0380067FB07E1E7D047CDE
:10918F0000E5FF5407F9F8121AE4E47B20FAF9F826
:10919F0012A64DC006C00790FE25E0FEA3E0FBAA75
:1091AF0006E4F9F8D007D00612A64DC3E49F90FE4F
:1091BF0029F074049E90FE28F04387807598509094
:1091CF00FE28E0F5BAA3E0F5AA75A101E5A1B40167
:1091DF000512ADC680037595037E007F127D007B5F
:1091EF00017AFC79CE12206090FE27E06002D2ACAB
:0191FF00224D
:10A3580090FE2A12ADB1A3ECF0A3EDF0E4FFFE7578
:10A36800A101E5A1B4010512ADC68003759503D31B
:10A3780090FE2EE09FEE6480F890FE2DE0648098B9
:10A38800401E90FE2A12ADBD8F828E8312177FF574
:10A3980099E59830E1FB5398FD0FBF00010E80CF7F
:01A3A8002292
:10B1510090FEF9EFF07B017AFE79F97D017C001216
:08B16100A35890FEF9E0FF2263
:10A8C30090FE2F12ADB1E4A3F0A3F090FE2F12ADD2
:10A8D300BDA3E0FEA3E0F5828E8312177FFF601312
:10A8E30012B15190FE33E004F070E090FE32E004C8
:0CA8F300F080D890FE32E0FEA3E0FF22CF
:10A4930090FBC712ADB190FBF27401F0A374FBF013
:10A4A300A374CAF090FBC7E0F9A3E0FAA3E090FE1F
:10A4B3001AC912ADB290FBF2E0F9A3E0FAA3E0905F
:10A4C300FE1DC912ADB212ADD312A57812ADD312CF
:0DA4D300B209AC06AD0712ADD312A358229A
:0300230002A2B284
:10A2B200C0E0C083C082C0D075D000C004C005C059
:10A2C20007E59830E02F90FCDEE0FF2401FDE43347
:10A2D200FCA3E06D7001EC601974CE2FF582E434BA
:10A2E200FCF583E599F090FCDEE004F0E0B41002A6
:10A2F200E4F05398FED007D005D004D0D0D082D05D
:04A3020083D0E032F2
:10AE28007FFF90FCDFE0FE90FCDEE06E601874CEE1
:10AE38002EF582E434FCF583E0FF90FCDFE004F0BB
:07AE4800E0B41002E4F02267
:10A2070090FE3412ADB1A3ECF0A3EDF0E4FDFCD366
:10A2170090FE38E09DEC6480F890FE37E06480980B
:10A22700402F12AE28EFF460F912ADBA8D828C83FD
:10A23700EF1217BEEFB40A12ED1D70011C12ADBA72
:10A247008D828C83E41217BE80070DBD00010C8040
:06A25700BEAE04AF0522BB
:108842004DFCBF000000FF000000000000F0E0004F
:1088520041FCBB0041FCBC0041FCCC0041FCCD0012
:0888620041FCBE0041FCBA001C
:109B1800C454F0FEEF4EFFF090FEE3E024BFF58260
:109B2800E434FCF58322E0FF90FEE4E022E0FE90BE
:109B3800FEEDE022E090FEE9FEE033333354F822F4
:109B480075A101E5A1640122E090FEE4FEE0C454A1
:109B5800F0FD22E0FD90FEEDE0FCED6C22E0FF243C
:109B6800FB24FB22C454F0FD90FCBAE05DFDEE221C
:109B780090FEEDE0FFEE6F2290FEE4E0540FF0A3BC
:109B8800E0FF22E0FEC454F05FFFEE4FF022F4FE47
:059B9800EF5EF0EE227B
:1067100090FEE4EDF0A3EBF090FEE3EFF01460499F
:106720001460791470030267C21470030267E124D5
:10673000FA700302681414700302685B240B600390
:106740000268C290FEE5E0FF700790FEE4E042FCC4
:1067500022EF90FEE4B40205E042C88004E0F45267
:10676000C890FEE4E0F452FC2290FEE5E0FF7007E2
:1067700090FEE4E042FD22EF90FCBBB40212129BBB
:106780002EFEEF4EFF90FCBB129B1FE05F42FD22EE
:10679000129B2E90FCBB129B9652FD2290FEE5E0D0
:1067A000FF700790FEE4E042FE22EF90FEE4B402A8
:1067B00005E042D88004E0F452D890FEE4E0F452C0
:1067C000FE2290FEE5E07012129B20C083C0821270
:1067D0009B2EFEEF4ED082D083F0129B20E0F5B0CE
:1067E0002290FEE5E0FF700790FEE4E042F322EF26
:1067F00090FCBCB40212129B2EFEEF4EFF90FCBC2C
:10680000129B1FE05F42F322129B2E90FCBC129B56
:106810009652F322129B807013129B20C083C08279
:10682000129B50EE4DD082D083F08028EF90FCCCAC
:10683000B4020E129B2E90FCCC129B18129B8B80E4
:1068400013129B2EC454F0F4FEEF5E90FCCC129B0E
:106850001FE05EF0129B20E0F58A2290FEE4E054F7
:106860001CF0A3E0FF7018129B20C083C082E09050
:10687000FEE4129B40FDEE4DD082D083F0803CEFD1
:1068800090FCCDB40220129B2E33333354F8FEEF2C
:106890004EFF90FCCD129B1FE0FE33333354F85F64
:1068A000FFEE4FF08015129B2E33333354F8F4FE75
:1068B000EF5E90FCCD129B1FE05EF0129B20E0F596
:1068C000C122129B48706E90FEE3129B6550072414
:1068D000FE602C0269EB12AEC390FEE5E0FF70078C
:1068E00090FEE4E0429B22EF90FEE4B40205E04219
:1068F0009C8004E0F4529C90FEE4E0F4529B2290D1
:10690000FEE5E0FF700790FEE4E0429722EF90FC86
:10691000BEB40212129B2EFEEF4EFF90FCBE129BE5
:106920001FE05F429722129B2EF4FEEF5E90FCBEAA
:10693000F0EE52972290FEE3E0FF24FA60331460F9
:1069400042146061240360030269EB90FEE5E0FEFF
:10695000700790FEE4E0429B22EE90FEE4B4020554
:10696000E0429C8004E0F4529C90FEE4E0F4529BF0
:106970002290FEE5E090FEE47004E0429422E0F410
:1069800052942290FEE5E0701574BF2F129B26C032
:1069900083C082129B2EFEEF4ED082D083F0129BDA
:1069A00020E0F59522129B807013129B20C083C0BB
:1069B00082129B50EE4DD082D083F08028EF90FC65
:1069C000BAB4020E129B2E90FCBA129B18129B8B2B
:1069D0008013129B2EC454F0F4FEEF5E90FCBA12AA
:0C69E0009B1FE05EF0129B20E0F5AD2252
:10AEC300EF24FA6011146012146013146014240444
:10AED3007013E4F5A12275A1012275A1022275A1C7
:06AEE300032275A1042208
:10947900AB05AA07EA14601914601B14601D146077
:109489001F24FA6020146022240B7023E5805BFFFF
:1094990022E5905BFF22E5A05BFF22E5B05BFF229E
:1094A900E5F25BFF22E58A5BFF22E5C15BFF221241
:1094B9009B487032EA24FB24FB500624FE600C8092
:1094C90047AF0212AEC3E59A5BFF22E58F5470FAEB
:1094D900758F7090FCBDE591F0E4F58FE04591F052
:1094E9008A8FE05BFF22EA24FA600F14601114608E
:1094F9001324037013E59A5BFF22E5935BFF22E5D2
:09950900955BFF22E5AD5BFF223A
:1078150090FEE8EFF0A3EDF090FEE8E0FF129B2468
:10782500E04DF0EF14602114603414603B146042A5
:1078350024FA605414607B240B60030278DE90FE0A
:10784500E8129B23E0F5802290FEE9E0FF90FCBB67
:10785500E05F42FD90FEE8129B23E0F5902290FE4A
:10786500E8129B23E0F5A02290FEE8129B23E0F5A9
:10787500B02290FEE9E0FF90FCBCE05F42F390FE91
:10788500E8129B23E0F5F22290FEE8E0FF129B242C
:10789500C083C082E090FEE9129B5490FCCCE05D71
:1078A500FDEE4DD082D083F074BF2F129B26E0F5FC
:1078B5008A2290FEE8E0FF129B24C083C082129BBF
:1078C5003CFD90FCCDE05DFDEE4DD082D083F074A3
:1078D500BF2F129B26E0F5C122129B48704390FEF4
:1078E500E8129B65500724FE601002797B12AEC337
:1078F50090FEE8129B23E0F59A2290FEE8E0FF1245
:107905009B24C083C082129B3CFD90FCBEE05DFDC4
:10791500EE4DD082D083F074BF2F129B26E0F591F7
:107925002290FEE8E0FF24FA601414601B14602224
:107935002403704274BF2F129B26E0F59A2290FE15
:10794500E8129B23E0F5932290FEE8129B23E0F5D5
:10795500952290FEE8E0FF129B24C083C082E0FEE2
:1079650090FEE9E0129B6C4DD082D083F074BF2F5E
:07797500129B26E0F5AD2294
:10797C0090FEEAEFF0A3EDF090FEEAE0FF129B24FC
:10798C00E0FEEDF4FDEE5DF0EF14602114603514B3
:10799C00603C14604324FA6056146077240B600337
:1079AC00027A4290FEEA129B23E0F5802290FEEAD6
:1079BC00129B23E0F59090FEEBE0FF90FCBBE05FA8
:1079CC00F452FD2290FEEA129B23E0F5A02290FED9
:1079DC00EA129B23E0F5B02290FEEA129B23E0F51D
:1079EC00F290FEEBE0FF90FCBCE05FF452F32290CF
:1079FC00FEEAE0FF129B24E0FEF58A74BF2F129B77
:107A0C0026C083C08290FEEBE0C454F0FF90FCCC07
:107A1C00027AD790FEEAE0FF129B24E0FEF5C174D7
:107A2C00BF2F129B26C083C08290FEEB129B41FF9E
:107A3C0090FCCD027AD7129B48703E90FEEA129BC6
:107A4C0065500724FE6010027AE212AEC390FEEA83
:107A5C00129B23E0F59A2290FEEAE0FF129B24E0B1
:107A6C00FEF59174BF2F129B26C083C08290FEEB53
:107A7C00129B41FF90FCBE805290FEEAE0FF24FA7C
:107A8C00601414601B1460222403704A74BF2F12FC
:107A9C009B26E0F59A2290FEEA129B23E0F59322B6
:107AAC0090FEEA129B23E0F5952290FEEAE0FF128D
:107ABC009B24E0FEF5AD74BF2F129B26C083C082C1
:107ACC0090FEEBE0C454F0FF90FCBAE05FF4FFEEE4
:077ADC005FD082D083F0228D
:1069EC0090FEEDEDF090FEECEFF014604414607648
:1069FC00147003026A93147003026AB424FA7003CD
:106A0C00026AE9147003026B3C240B6003026B8E68
:106A1C0090FEECE0FF129B24C083C082129B35FDDC
:106A2C00EE6DD082D083F074BF2F129B26E0F580E0
:106A3C002290FEECE0FF129B24129B35FDF4FCEE41
:106A4C005CF59090FCBBE05D62FD74BF2F129B2641
:106A5C00C083C082129B78D082D083F090FEEC125F
:106A6C009B23E0F5902290FEECE0FF129B24C08368
:106A7C00C082129B35FDEE6DD082D083F074BF2F97
:106A8C00129B26E0F5A02290FEECE0FF129B24C0A6
:106A9C0083C082129B35FDEE6DD082D083F074BF23
:106AAC002F129B26E0F5B02290FEECE0FF129B2407
:106ABC00129B35FDF4FCEE5CF5F290FCBCE05D62E3
:106ACC00F374BF2F129B26C083C082129B78D08296
:106ADC00D083F090FEEC129B23E0F5F22290FEECBA
:106AEC00E0FF129B24129B35F4FDEE5DF58A74BF1A
:106AFC002F129B26C083C08290FEEDE0C454F0FFA1
:106B0C0090FCCCE05FFFEE6FD082D083F090FEEC77
:106B1C00E0FF129B24C083C082129B35540FFDEE04
:106B2C006DD082D083F074BF2F129B26E0F58A22A1
:106B3C0090FEECE0FF129B24129B35F4FDEE5DF50C
:106B4C00C174BF2F129B26C083C08290FEED129B96
:106B5C0041FF90FCCDE05FFFEE6FD082D083F090D0
:106B6C00FEECE0FF129B24C083C082129B35541CA8
:106B7C00FDEE6DD082D083F074BF2F129B26E0F512
:106B8C00C122129B48706890FEEC129B6550072442
:106B9C00FE6027026CA412AEC390FEECE0FF129BC9
:106BAC0024C083C082129B35FDEE6DD082D083F061
:106BBC0074BF2F129B26E0F59A2290FEECE0FF1298
:106BCC009B24129B35FDF4FCEE5CF59190FCBEE031
:106BDC005D629774BF2F129B26C083C082129B7874
:106BEC00D082D083F090FEEC129B23E0F5912290A2
:106BFC00FEECE0FF24FA602B146046146061240361
:106C0C006003026CA490FEECE0FE129B24C083C0D7
:106C1C0082129B5BD082D083F074BF2E129B26E035
:106C2C00F59A2290FEECE0FE129B24C083C08212E7
:106C3C009B5BD082D083F074BF2E129B26E0F59321
:106C4C002290FEECE0FE129B24C083C082129B5B60
:106C5C00D082D083F074BF2E129B26E0F59522745F
:106C6C00BF2F129B26C083C082129B35129B6C6D6A
:106C7C00D082D083F074BF2F129B26C083C082E0D9
:106C8C00FF90FEEDE0540FFEEF6ED082D083F090BB
:096C9C00FEEC129B23E0F5AD2291
:10B16900786DE6FF90FF8093FE74802FF582E434BA
:08B17900FFF583EEF006E6226B
:10B1C700C3EE940240037FFF2274002FF58274EED2
:07B1D7003EF583E493FF2223
:10A3A90090FEEEEEF0A3EFF0C3EE940250407480FD
:10A3B9006480700374FFF4703530AF02D230C2AFDD
:10A3C90090FEEFE0240090FEEEE034EEF5F9A3E014
:10A3D900F5FA786D764012B169B480FAAF05786DF7
:0FA3E900A6077B01796D12FFC0303002D2AF2280
:10AD5E0074806480700374FFF4701E30AF02D230C2
:10AD6E00C2AF75F9EEE4F5FA786DF612B169B4403A
:0AAD7E00FA12FF80303002D2AF223B
:0C886A00C13141FE650043FE66000000C5
:10B0D00090FE66E0FBA3E0FAA3E0F9EA494B229078
:0CB0E000FE66A3E0FAA3E0F5828A83225A
:10A9390075A101E5A1B4011BEF24FE600C14600EA2
:10A949002403702375A49C801E75A4DC801975A44A
:10A95900FC801443F580EF24FE6009240270087519
:0AA96900A4B8800375A4F8D2BD2243
:0CB3490090FE66EBF0A3EAF0A3E9F0220E
:10AE4F0030310CEF70037F862290FE65E0FF227594
:10AE5F00A101E5A1B40107EF04F5A6AFA722EF709A
:07AE6F0003AFA622AFA722EA
:03006B00029E07EB
:109E0700C0E0C0F0C083C082C0D075D000C000C021
:109E170001C002C003C004C005C006C007C2317537
:109E2700A101E5A164017019F5A612B0D0602AE579
:109E3700A530E6047F0180027F0012B0DFADA78066
:109E47001512B0D06013E5A530E6047F0180027FCC
:109E57000012B0DF7D10121CDE43A580D007D006AC
:109E6700D005D004D003D002D001D000D0D0D0820A
:079E7700D083D0F0D0E032EF
:0688760041FEFA01C132CF
:06B3A90090FEFAEFF02215
:10B18100EF6005D232758680E5FFB430037F01227E
:08B1910075FF30D2AF7F0022F0
:08B39300303204D2AED2BE221A
:10594500444247434D4420537472696E6720427543
:10595500666665722046756C6C0D0A0025732025F8
:105965005820255820255820255800627573004475
:105975004247434D44206275733A204275733D306A
:105985007825302E32582C20506F72743D30782592
:10599500302E32582C2053706565643D30782530A3
:1059A5002E32580D0A0063697200444247434D4444
:1059B500206369723A20436F64653D307825302E47
:1059C50032580D0A0077723000444247434D442057
:1059D5007772303A2049443D307825302E32582CA4
:1059E500205265673D307825302E32582C20446191
:1059F50074613D307825302E32580D0A00726430BE
:105A050000444247434D44207264303A2049443DA6
:105A1500307825302E32582C205265673D30782558
:105A2500302E32582C20446174613D003078253089
:105A35002E32580D0A0074623000444247434D44EB
:105A4500207462303A2049443D307825302E325852
:105A55002C205265673D307825302E32582C204D4C
:105A650061736B3D307825302E32582C204461749B
:105A7500613D0063623000444247434D4420636208
:105A8500303A2049443D307825302E32582C20526A
:105A950065673D307825302E32582C204D61736B6B
:105AA5003D307825302E32582C20446174613D00FC
:105AB50077723100444247434D44207772313A2092
:105AC50049443D307825302E32582C205265673DAB
:105AD500307825302E32582C20446174613D307861
:105AE50025302E32580D0A00726431004442474376
:105AF5004D44207264313A2049443D307825302E9A
:105B050032582C205265673D307825302E32582C7E
:105B15002053697A653D307825302E32582C204443
:105B25006174613D002852656164206E756D626522
:105B350072206578636565642061206D6178206FEA
:105B45006620256420627974657329000D0A00209A
:105B550000307825302E32582C20007462310044F4
:105B65004247434D44207462313A2049443D3078E0
:105B750025302E32582C205265673D307825302E41
:105B850032582C204D61736B3D307825302E3258BC
:105B95002C20446174613D006362310044424743F7
:105BA5004D44206362313A2049443D307825302EFA
:105BB50032582C205265673D307825302E32582CCE
:105BC500204D61736B3D307825302E32582C2044A2
:105BD5006174613D0077723200444247434D442071
:105BE5007772323A2049443D307825302E32582C90
:105BF500205265673D307825302E34582C2044617D
:105C050074613D307825302E32580D0A00726432A9
:105C150000444247434D44207264323A2049443D92
:105C2500307825302E32582C205265673D30782546
:105C3500302E34582C2053697A653D307825302E26
:105C450032582C20446174613D0074623200444234
:105C550047434D44207462323A2049443D3078250B
:105C6500302E32582C205265673D307825302E3441
:105C7500582C204D61736B3D307825302E32582CD1
:105C850020446174613D0063623200444247434DE4
:105C950044206362323A2049443D307825302E3223
:105CA500582C205265673D307825302E34582C20ED
:105CB5004D61736B3D307825302E32582C20446170
:105CC50074613D004552524F523A2049494320667E
:105CD50061696C65642025642C20494943416464ED
:105CE500723D307825302E32582C2052656741643C
:0D5CF50064723D307825302E32580D0A00C3
:08887C0041FCB50041FCB30012
:1073420078A17CFC7D017BFF121E99EF2278A17C43
:10735200FC7D017BFF121E99EF22A3F090FC9AE0C4
:10736200FF90FC9DE0FCA3E090FD5EFD7B017AFCBA
:1073720079A1E4F0A304F02278A17CFC7D017BFFDB
:10738200121E99EF2278A17CFC7D017BFF121E99CF
:10739200EF227BFF7A5B795690FCB7E024A1F5825D
:1073A200E434FCF583E0FFE490FBCAF0A3EFF022A3
:1073B20078A17CFC7D017BFF121E99EF2290FCA13B
:1073C200F090FC9AE0FF90FC9CE0FD7B017AFC7956
:1073D200A12278A17CFC7D017BFF121E99EF2290F5
:1073E200FC9CE0FEA3E04EF0A3E0F022E4F0A374E4
:1073F20012F07BFF7A5B792A90FBCAE4F0A3741245
:10740200F0227BFF7A5A793190FCA1E0FF90FBCA0F
:10741200E422F0A3EDF0A3EBF0A3EAF0A3E9F090ED
:10742200FCB6E4F0A3740AF0E4A3F0A3F02290FC0B
:107432009CE0FD90FC9EE0FB22FDE0FBA3E0FAA3B2
:10744200E0F9A3E0FFA3E090FCF2CFF0A3EFF0EDB0
:1074520022A3F0A37401F0A322A3F0A37422F043A9
:10746200FF407AFF7980121CDA53FFBF22E0FEA3AD
:10747200E0FF90FCB6E0FCA3E0FDC39FEC9E22E09F
:10748200FFE490FBCCF0A3EFF022D390FCB7E094A2
:107492000090FCB6E0940022C390FCB9E094039003
:1074A200FCB8E09400227BFF90FC99E0FFA3E0226D
:1074B20078A17CFC7D017BFF121E99EF22E054FE35
:1074C200FD7B0190FCF2E4F0A322A3E024FDF09006
:1074D200FCB6E034FFF02290FCF4EFF090FCB3E055
:1074E200FF227BFF7A5B79512290FCA1E0FF90FCA6
:0D74F2009EE02290FCA1E0FF90FCA0E022B3
:1040A40012AE2890FEFBEFF0F47003024467E0FFC9
:1040B40090FCB5E0FE04F074A12EF582E434FCF526
:1040C40083EFF090FCB5E0D39412400E7BFF7A5955
:1040D400794512A493E490FCB5F090FEFBE0FF64F4
:1040E4000A6008EF640D6003024467E490FCB5F0D5
:1040F40090FBF874FFF0A37459F074611274537454
:10410400FFF0748012745374FCF0A3749912745405
:1041140074FCF0A3749B12745474FCF0A3749D1289
:10412400745474FCF0A3749FF01273CD126477E49A
:1041340090FCA4F07A597970127342701D7A5979FF
:104144007412446D90FC9AE0FF12743012AA179016
:10415400FC9AE090FCB3F00244677A5979AB12738D
:1041640042703F7A5979AF1274A8CF1273AA12A47D
:1041740093D23190FC9AE090FE65F090FE66E0FBED
:10418400A3E0FAA3E0F9EA494B700302446790FE06
:1041940066A3A3E0F5828A837D10E4FF121CDE028D
:1041A40044677A5979CA12734F70127A5979CE12C8
:1041B400446D1274307F7512B30C0244677A5A79D5
:1041C4000212734F70207A5A79061274A890FBCAAF
:1041D400CFF0A3EFF090FC9BE0FFA3E0CF12748438
:1041E40012A49302421C7A5A793B12737A70117AA0
:1041F4005A793F1244A01274307F6312B30C8018B2
:104204007A5A797812737A70337A5A797C1244A084
:104214001274307F5312B30C90FC9CE0FF12B280F6
:1042240090FC9FE4F0A3EFF07BFF7A5A793190FC85
:104234009FE0FFA3E090FBCACF0244287A5A79B5E5
:1042440012738770247A5A79B91244D390FC9EE091
:1042540090FCA1F090FC9AE0FF90FC9CE090FDA5FE
:1042640012736D1295A90244677A5A79ED12738715
:1042740070777A5A79F11244D3D390FC9EE0941269
:1042840090FC9DE0940040061273EE12A49390FCFF
:104294009AE04401FFC0071273C8A3E0FFA3E090B3
:1042A400FDA5CFF0A3EFF0D0071295A9EF600302AC
:1042B400446790FCB6F0A3F090FC9D12746F5026F6
:1042C400ED540F70061274E412A49390FCB7E054FA
:1042D4000770031245E31273941245ED70DA90FCF3
:1042E400B6E004F080D20243F77A5B79601273B2CD
:1042F40070277A5B79641245891295A9EF600302ED
:1043040044671274EBFEEF6E1273BF1245D660035E
:104314000244671274040244287A5B799D1273B2D2
:1043240070287A5B79A11245891295A9EF6003027E
:1043340044671274EBF4FEEF5E1273BF1245D6604D
:10434400030244671274040244287A5B79DA127314
:10435400D470171273E17A5B79DE12450690FCA0E3
:10436400E012735C12933E0244677A5C7912127312
:10437400D460030243FD1273E17A5C791612450698
:10438400D390FCA0E0941290FC9FE09400400612AD
:1043940073EE12A49390FC9AE04401FFC00790FCD2
:1043A4009DE0FCA31273CBA3E0FFA3E090FD5ECFDE
:1043B400F0A3EFF0D00712933EEF6003024467903E
:1043C400FCB6F0A3F090FC9F12746F5026ED540FCE
:1043D40070061274E412A49390FCB7E054077003BF
:1043E4001245E31273941245ED70DA90FCB6E004C2
:1043F400F080D21274E40244647A5C794F1274B28D
:1044040070291273E17A5C795312453912933EEFA5
:1044140070511274F5FEEF6E12735C12933EEF70DE
:1044240042127404F0A3EFF00244647A5C798C12B3
:1044340074B2702F1273E17A5C7990124539129339
:104444003EEF701F1274F5F4FEEF5E12735C12936C
:104454003EEF700F7BFF7A5A793190FCA11273A75B
:1044640012A49390FEFBE0FF227BFF90FC99E0FFF7
:10447400A3E090FBCACFF0A3EFF090FC9BE0FFA376
:10448400E090FBCCCFF0A3EFF090FC9DE0FFA3E025
:1044940090FBCECFF0A3EFF012A493227BFF90FC0D
:1044A40099E0FFA3E090FBCACFF0A3EFF090FC9B50
:1044B400E0FFA3E090FBCCCFF0A3EFF090FC9DE0F5
:1044C400FFA3E090FBCECFF0A3EFF012A493227BE6
:1044D400FF90FC99E0FFA3E090FBCACFF0A3EFF0BC
:1044E40090FC9BE0FFA3E090FBCCCFF0A3EFF09017
:1044F400FC9DE0FFA3E090FBCECFF0A3EFF012A46D
:1045040093227BFF90FC99E0FFA3E090FBCACFF0DD
:10451400A3EFF090FC9DE0FFA3E090FBCCCFF0A3D1
:10452400EFF090FC9FE0FFA3E090FBCECFF0A3EF71
:10453400F012A493227BFF90FC99E0FFA3E090FB90
:10454400CACFF0A3EFF090FC9DE0FFA3E090FBCC7A
:10455400CFF0A3EFF090FC9FE0FFA3E090FBCECF61
:10456400F0A3EFF012A49390FC9AE04401FF90FCB6
:104574009DE0FCA3E0FD7B017AFC79A190FD5EE463
:10458400F0A304F0227BFF90FC99E0FFA3E090FBF2
:10459400CACFF0A3EFF090FC9BE0FFA3E090FBCC2C
:1045A400CFF0A3EFF090FC9DE0FFA3E090FBCECF13
:1045B400F0A3EFF012A49390FC9AE04401FF90FC66
:1045C4009CE0FD7B017AFC79A190FDA5E4F0A304B5
:1045D400F02290FDA5E4F0A304F01295A9EF227B4C
:1045E400FF7A5B795412A4932212A49390FCB7E04F
:0345F40004F022AE
:1095A90090FDA0EF12741490FCB3E0FF90FDA07A37
:1095B900FD79A11274BF04F0A3F01274FF90FCB4FA
:1095C900EFF0E0FEC00690FDA0E090FDA212743B12
:1095D90030E0047F0080027F021274D91274FFD038
:1095E900E04F90FCB4F0602390FCB7E0FF12B32584
:1095F90012748C40031274CC90FCB9E004F070062C
:1096090090FCB8E004F012749A409C90FCB4E0FF1E
:10961900601F7BFF7A5C79C91273A990FDA012744F
:109629008190FDA1E0FF90FBCEE4F0A3EFF012A43E
:079639009390FCB4E0FF2256
:10933E0090FD58EFF0A3EC12741490FCB3E0FF9084
:10934E00FD587AFD79591274BF7402F0A314F0120D
:10935E0074FF90FCB4EFF0E0FEC00690FD58E09074
:10936E00FD5B12743B30E0047F0080027F021274BA
:10937E00D91274FFD0E04F90FCB4F0602390FCB78C
:10938E00E0FF12B32512748C40031274CC90FCB91A
:10939E00E004F0700690FCB8E004F012749A409A63
:1093AE0090FCB4E0FF60217BFF7A5C79C91273A94F
:1093BE0090FD5812748190FD59E0FFA3E090FBCE12
:0E93CE00CFF0A3EFF012A49390FCB4E0FF22C6
:10B2800090FF807485F0A3EFF0746E12745B786E9B
:03B29000E6FF22B4
:0DB30C0090FF80EFF0A3EDF0EB12745B22D8
:0E88840043FA8C01FA9641FA900041FA8F00F7
:1084830090FE14E0FBA3E0FAA3E0F92290001FE4BE
:10849300F5F012197A90001502177FE0FEA3E0FFB2
:1084A3007C007D051217E090FA8CE0FBA3E0FAA3B1
:1084B300E02FF9EA3EA801FCAD037B017AFF798046
:1084C3002290001FE4F5F012197A900016021C2B7B
:1084D30090FA90E0FFC390FA95E09F7480F890FAC9
:1084E30094E06480982290001FE475F0011218E173
:1084F300FEC3E5F02290FA90E075F005A4FF90FA30
:108503008CE0FBA3E0FAA3E022EBF0A3EAF0A3E9FB
:10851300F022FD7401F0A374FFF0A37480F02290A5
:10852300000402177F7E007F0512174090FA90E047
:1085330004F0227F057E0012203CEF2290FA90E0A7
:108543004480F02290001FE4F5F002197A2404F924
:06855300E43AFA0217668B
:1045F70090FE1412850C900006121C2B90FE1712C9
:10460700850C12848312176624F9B407004003024D
:104617004B2790462775F003A4C58325F0C5837300
:1046270002463C0247030248B602490C02496502AA
:1046370049DF024A7B90FE1712848612852230E1F9
:10464700751284831284CDC003C002C00112848313
:10465700128498FDD001D002D00312AF5112848387
:104667001284E99432EE94005003024B2712848F90
:10467700FF1284BD128D48EF602A128483128522AF
:1046870030E0191284CDC003C002C0011284831226
:104697008498FDD001D002D00312AFB41284837482
:1046A70008024B24128483128498FFE4FD12AD881C
:1046B70090FE140248F012848312852230E019120A
:1046C70084CDC003C002C001128483128498FDD038
:1046D70001D002D00312AFB41284831284CDC00379
:1046E700C002C001128483128498FDD001D002D089
:1046F7000312AF721284837405024B24128483124F
:104707008498FFE4FD12AD88128483128498124BBB
:104717002890FE1430E61E1284861284CDC003C092
:1047270002C001128483128498FDD001D002D00305
:1047370012AFD5801C1284861284CDC003C002C07C
:1047470001128483128498FDD001D002D00312AFE6
:10475700F6E490FF88F012A4E07C017D0012184770
:1047670090FF88E02480F582E434FFF583EDF09034
:10477700FF88E004F0E0C3940840DB1284831284CE
:10478700CDC003C002C00112848312849890FD73C8
:10479700128515D001D002D00312AC071284831200
:1047A7008498FF1284BD12ADDA1284831284CDC0BF
:1047B70003C002C00112848312849890FD7A128587
:1047C70015D001D002D0031290BAEF70241284835F
:1047D7001284CDC003C002C001128483128498FDE5
:1047E700D001D002D00312B0571284837407024B52
:1047F70024128483128498FF1284BD12AE0112849E
:1048070083128498FF1284BD128D48EF702412849E
:10481700831284CDC003C002C0011284831284981E
:10482700FDD001D002D00312B0571284837407025F
:104837004B241284831284CDC003C002C0011284AA
:1048470083128498FD90FD81128516D001D002D085
:104857000312AC33128483900019121C2BE94A4BC4
:10486700704590FA90E0C394085039E490FA94F0B8
:10487700A3F01284D3501812849E128536601090CC
:10488700FA95E004F070EB90FA94E004F080E312FC
:1048970084D340131284F82FF9EA35F01284B81242
:1048A7008528800312853F1284837409024B2412E2
:1048B70084831284E99407EE94005003024B271275
:1048C70084CDC003C002C001128483128498FDD036
:1048D70001D002D00312ACE0EF90FE14600B1284FB
:1048E70086128547740A024B241284861284CDC02F
:1048F70003C002C001128483128498FDD001D00244
:10490700D00302B057128483129F52EF7031128482
:10491700831284E9940AEE94005003024B27128411
:10492700C4C003C002C001128483128498FDD00161
:10493700D002D00312B0571284837407024B24129B
:10494700848312848F124B2890FE1430E608128459
:1049570086740D024B24128486740B024B24E49058
:10496700FF80F01284831284CD12B2E3EF700C90B3
:10497700FF80E004F0E0C394FA40E8E490FF81F0A0
:104987001284831284CD12B2E3BF010C90FF81E041
:1049970004F0E0C394FA40E81284831284CDC00384
:1049A700C002C001128483128498FDD001D002D0C6
:1049B7000312AF931284831284CDC003C002C001D7
:1049C700128483128498FDD001D002D00312AF72F3
:1049D700128483740C024B2490FE1712848612856E
:1049E7002230E16C1284831284E9944BEE940050D8
:1049F70003024B27128547129F52EF70451284839B
:104A070012852230E2211284CDC003C002C00112F8
:104A17008483128498FDD001D002D00312B03712DC
:104A270084837407024B2490FE1412850412855068
:104A370044041217AC12848390001FE475F032020D
:104A4700197A90FE1412850412855054FB024B24E8
:104A57001284831284CDC003C002C0011284831262
:104A67008498FDD001D002D00312B037128483742A
:104A770007024B24128483128498FF12B07790FAAE
:104A870091EFF030E56C12848312848FFF1284BD9E
:104A970012A97390FF80E0FD20E71CA3E0FF20E34D
:104AA7001612848390FD64EFF0127C43EF602012AE
:104AB7008483740B024B2490FF80E030E703128558
:104AC7003F90FF81E030E30790FA8FE04408F0124F
:104AD70084831284CDC003C002C001128483128470
:104AE70098FDD001D002D00312B057128483740707
:104AF700802B1284831284E994FAEE9400402112E9
:104B070084C4C003C002C001128483128498FDD0FC
:104B170001D002D00312B05712848374071217AC66
:0B4B270022FF12B07790FA91EFF0220D
:109F520090FDA712850C1284CDC003C002C00190EF
:109F6200FDA7128486128498FD90FD887401F0A3E7
:109F720074FDF0A374AAF0D001D002D00312A5C2DE
:109F8200EF7002FF2290FDA7128486128498FF7B55
:109F9200017AFD79AC12A085EF7002FF2290FDAC30
:109FA200E0FEA3E0FF90FDAAE0B50608A3E0B50736
:079FB200037F01227F002262
:107C430090FD6012850CA3EDF0A3E0540FFF90FAB2
:107C53008FE0FEEFD39E40028002AF0690FA8FEFD3
:107C6300F012A84AE490FA92F0A3F090FD63E0FFCB
:107C730090FA92E0FCA3E0FDC39F7480F8EC64806B
:107C8300984003027D0990FD60128486128498FF58
:107C93001284BD90FDE2EDF090FD63E090FDE3F012
:107CA300127EDAEF7002FF2290FA90E0C39408503C
:107CB30039E490FA94F0A3F01284D3501812849EFE
:107CC300128536601090FA95E004F070EB90FA9408
:107CD300E004F080E31284D340131284F82FF9EA0E
:107CE30035F01284B8128528800312853F1284BDB3
:107CF3007D0512901390FA93E004F0700690FA92C7
:107D0300E004F0027C6E90FD63E0701890FD601259
:107D13008486128498FF1284BDE490FDE2F0A304EC
:107D2300F0127EDA90FD63E090FF80F090FD64E056
:107D330090FF81F090FD601284861284CDC003C051
:107D430002C00190FD60128486128498FD90FD8F1D
:107D53007401F0A374FFF0A37482F0D001D002D0B9
:107D63000312AD0A1284BD7D0A1290131282C590CC
:107D7300FD6512850C90FD60128486128498FF12B3
:107D830084BD12A9AA90FD65128504F8AC02128481
:0E7D9300BB7F1412853860037F00227F01221F
:0688920043FBAD01FFC035
:1088990090FBBBE0FCA3E0FDA3E0FEA3E0FF90FB9F
:1088A900B7E0F8A3E0F9A3E0FAA3E022121BEE90E7
:1088B900FD19E0FCA3E0FDA3E0FEA3E0FF227E009A
:1088C9007F407D0090FBADE0FBA3E0FAA3E022EB43
:1088D9002FFFEA3EFEE93DFDE83CFC22F9A3E05406
:1088E9000F75F004A4F58285F08322EF4BFFEE4A61
:1088F900FEED49FDEC48FC226FFFEA6EFEE96DFDD5
:10890900E86CFC225FFFEA5EFEE95DFDE85CFC22A3
:1089190090FD15C9F0A3EAF0A3E9F07B017AFB7990
:108929009622EF6BFFEE6AFEED69FDEC68FC229082
:10893900FD19021BEE121B5B90FD1222F074982B9D
:10894900F58274FB3AF5832274972BF58274FB3A0E
:0D895900F58322F9122060E490FBAAF022C1
:10A84A0090FB96121BFA6745230190FB9A121BFA9A
:10A85A00EFCDAB8990FB9E121BFA98BADCFE90FBF7
:10A86A00A2121BFA1032547690FBA6121BFAC3D21C
:0DA87A00E1F01288C712895CA3F0A3F02260
:1090130090FE69EBF0A3EAF0A3E9F0A3EDF0FF9073
:10902300FBACE02FF090FBABE03400F090FE6CE083
:10903300FF70030290B990FBAAE0FEC374409EFE4A
:10904300C39F5004AF06800590FE6CE0FF90FBB019
:10905300EFF07E001288CDF990FBAAE0FD7C00E9D9
:109063002DF9EC3AA801FCAD0390FE691288D0F902
:1090730012174090FBB0E0FF90FBAAE02FF090FEA8
:109083006AE48FF012187D90FE6CE0FF90FBB0E075
:10909300FEC3EF9E90FE6CF090FBAAE0C3944040A9
:1090A3008B90FBAD1288AD128919125D021288C72D
:0790B30012895C02902F22DC
:1082C5001288CDF990FBAAE0FF04F08F8275830038
:1082D50074801217BE90FBAAE0FFC374409FC3943D
:1082E5000250071288C7F912206090FBABE0FEA38D
:1082F500E07803C333CE33CED8F9F0EE90FBABF084
:10830500E0FF1288CDF990003EEF1217BE90FBAC4E
:10831500E090003F1217BE90FBAD1288AD1289198F
:10832500125D02E490FBB1F0A3F0C390FBB2E094C0
:108335001490FBB1E0648094805066E0FEA3E0FFFA
:108345002496F58274FB3EF583E0FD90FF80F07482
:10835500992FF58274FB3EF583E0FF90FBB1E0FABF
:10836500A3E0FB2496F58274FB3AF583EFF074994C
:108375002BF58274FB3AF583EDF0128951E0FF90FD
:10838500FF80128945E0FE128951EE128945EFF012
:1083950090FBB2E02404F090FBB1E03400F00283DE
:0583A5002F12892422C3
:105D020090FD12EBF0A3EAF0A3E9F0121B0B90FB5B
:105D1200B3121BEE900004121B2B90FBB7121BEE6A
:105D2200900008121B2B90FBBB121BEE90000C1272
:105D32001B2B90FBBF121BEE900010121B2B90FB33
:105D4200C3121BEEE490FD18F090FD18E0FFD3940F
:105D52004F4003025FEEEFC394105003025DEA90DE
:105D6200FD151288D0F9A3E024081288E8121B2B33
:105D7200C00790FD15A3A3A3E0240D1288E8121B0F
:105D8200B2D007EB128901C00790FD151288D0F935
:105D9200A3E024021288E8121BB2D00712892BC09A
:105DA2000790FD151288D01288E5121BB2D0071297
:105DB200892B90FD191288B57801121AF8C004C017
:105DC20005C006C0071288B8781F121AD1D003D0B6
:105DD20002D001D0001288F4C00790FD151288D0BD
:105DE2001288E5D007121B7590FD151288D0128813
:105DF200E5121B2B12893890FD191288AAFBC000EC
:105E0200C001C002C00390FBB31288BB7805121A0E
:105E1200F8C004C005C006C00790FBB31288BB7867
:105E22001B121AD1D003D002D001D0001288F4D0B4
:105E320003D002D001D0001288D812893890FD1800
:105E4200E0D394135048A31288AAFBC000C001C03B
:105E520002C00390FBB71288BB121AC490FBBF1298
:105E620088AA12890DC004C005C006AB0712889922
:105E720012890DD002D001D0001288F4EF2499FFCC
:105E8200EE3479FEED3482FDEC345A025F6C90FD03
:105E920018E0D39427502EA31288AAFBC000C00199
:105EA200C002C00312889912890190FBBF1288AA0E
:105EB200128901EF24A1FFEE34EBFEED34D9FDECA3
:105EC200346E025F6C90FD18E0D3943B506FA312C6
:105ED20088AAFBC000C001C002C00390FBBF1288A9
:105EE2009C12890DC004C005C006AB07A31288BB73
:105EF20090FBB7A3A3A3E012890DD002D001D0007A
:105F02001288F4C004C005C006AB0790FBBF12881C
:105F1200BB90FBBB1288AA12890DD002D001D0001F
:105F2200EB4FFFEA4EFEE94DFDE84CFCEF24DCFFAF
:105F3200EE34BCFEED341BFDEC348F802D90FD1948
:105F42001288AAFBC000C001C002C00312889912C5
:105F5200890190FBBF1288AA128901EF24D6FFEEB5
:105F620034C1FEED3462FDEC34CAFCD003D002D061
:105F720001D0001288D81289381288B890FBC31257
:105F820088AAFBEF2BFFEE3AFEED39FDEC38FC124E
:105F9200893890FBBF1288BBA3121BEE90FBBB1289
:105FA20088BBA3121BEE90FBB71288BB781E121A95
:105FB200F8C004C005C006C00790FBB71288BB78C2
:105FC20002121AD1D003D002D001D0001288F4A359
:105FD200121BEE90FBB31288BBA31288B590FBB3E1
:105FE200121BEE90FD18E004F0025D4B90FD1212C0
:105FF20088D0F9C002C001121B0B90FBB31288AA11
:106002001288D9D001D00212893E1288D02404F914
:10601200E43AFAC002C001121B0B1288A71288D9F7
:10602200D001D00212893E1288D02408F9E43AFA4B
:10603200C002C001121B0B90FBBB1288AA1288D9A6
:10604200D001D00212893E1288D0240CF9E43AFA27
:10605200C002C001121B0B90FBBF1288AA1288D982
:10606200D001D00212893E1288D02410F9E43AFA03
:10607200C002C001121B0B90FBC31288AA1288D95E
:07608200D001D002021B5BFC
:0300000002975D07
:0C975D00787FE4F6D8FD75816E0297A4B9
:10167000E709F608DFFA8046E709F208DFFA803E5C
:1016800088828C83E709F0A3DFFA8032E309F60849
:10169000DFFA8078E309F208DFFA807088828C83B1
:1016A000E309F0A3DFFA806489828A83E0A3F60865
:1016B000DFFA805889828A83E0A3F208DFFA804C3F
:1016C00080D280FA80C680D4806980F28033801016
:1016D00080A680EA809A80A880DA80E280CA80337F
:1016E00089828A83ECFAE493A3C8C582C8CCC583F7
:1016F000CCF0A3C8C582C8CCC583CCDFE9DEE780C7
:101700000D89828A83E493A3F608DFF9ECFAA9F045
:10171000EDFB2289828A83ECFAE0A3C8C582C8CC9B
:10172000C583CCF0A3C8C582C8CCC583CCDFEADEB4
:10173000E880DB89828A83E493A3F208DFF980CC16
:1017400088F0EF60010E4E60C388F0ED2402B4040F
:101750000050B9F582EB2402B4040050AF232345B6
:0617600082239016C07305
:10176600BB010689828A83E0225002E722BBFE0281
:09177600E32289828A83E49322B4
:10177F00BB010CE58229F582E5833AF583E022501F
:10178F0006E92582F8E622BBFE06E92582F8E22269
:0D179F00E58229F582E5833AF583E4932283
:1017AC00BB010689828A83F0225002F722BBFE011C
:0217BC00F32216
:1017BE00F8BB010DE58229F582E5833AF583E8F061
:1017CE00225006E92582C8F622BBFE05E92582C80D
:0217DE00F222F5
:1017E000EF8DF0A4A8F0CF8CF0A428CE8DF0A42E1D
:0217F000FE22D7
:1017F200BC000BBE0029EF8DF084FFADF022E4CCDB
:10180200F875F008EF2FFFEE33FEEC33FCEE9DECA3
:10181200984005FCEE9DFE0FD5F0E9E4CEFD22EDE9
:10182200F8F5F0EE8420D21CFEADF075F008EF2F33
:10183200FFED33FD4007985006D5F0F222C398FD24
:051842000FD5F0EA22C1
:10184700C2D5EC30E709B2D5E4C39DFDE49CFCEEBC
:1018570030E715B2D5E4C39FFFE49EFE1217F2C32B
:10186700E49DFDE49CFC80031217F230D507C3E426
:061877009FFFE49EFE222B
:10187D00C5F0F8A3E028F0C5F0F8E58215827002F6
:06188D001583E038F02293
:10189300A3F8E0C5F025F0F0E58215827002158308
:0618A300E0C838F0E82265
:1018A900BB0110E58229F582E5833AF583E0F5F07D
:1018B900A3E0225009E92582F886F008E622BBFE5A
:1018C9000AE92582F8E2F5F008E222E5832AF583A0
:0818D900E993F5F0A3E9932265
:1018E100BB010FF8E58229F582E5833AF583E80229
:1018F10018935011C58229F808C5F026C6F5F018CD
:10190100C58236C622BBFE15C58229F808E2C5F09C
:1019110025F0F218E2C5823582F2E58222E5832ABA
:0C192100F583E993F5F0A3E993C5F022EB
:10192D00BB010DC58229C582C5833AC58302187DC9
:10193D005011C58229F808E5F026F618F5F0E58274
:10194D0036F622BBFE11C58229F808E225F0F5F026
:10195D00F218E23582F222F8E58229F582E5832A32
:0D196D00F58374019325F0F5F0E493382222
:10197A00F8BB0111E58229F582E5833AF583E8F09F
:10198A00E5F0A3F0225009E92582C8F608A6F0225C
:0D199A00BBFE09E92582C8F2E5F008F22243
:1019A700E88FF0A4CC8BF0A42CFCE98EF0A42CFCDF
:1019B7008AF0EDA42CFCEA8EF0A4CDA8F08BF0A45D
:1019C7002DCC3825F0FDE98FF0A42CCD35F0FCEBBC
:1019D7008EF0A4FEA9F0EB8FF0A4CFC5F02ECD3981
:0F19E700FEE43CFCEAA42DCE35F0FDE43CFC22EE
:1019F60075F008758200EF2FFFEE33FECD33CDCCA8
:101A060033CCC58233C5829BED9AEC99E58298402A
:101A16000CF582EE9BFEED9AFDEC99FC0FD5F0D607
:101A2600E4CEFBE4CDFAE4CCF9A88222B800C1B931
:101A36000059BA002DEC8BF084CFCECDFCE5F0CB6F
:101A4600F97818EF2FFFEE33FEED33FDEC33FCEBA8
:101A560033FB10D703994004EB99FB0FD8E5E4F963
:101A6600FA227818EF2FFFEE33FEED33FDEC33FC50
:101A7600C933C910D7059BE99A4007EC9BFCE99A44
:101A8600F90FD8E0E4C9FAE4CCFB2275F010EF2F89
:101A9600FFEE33FEED33FDCC33CCC833C810D70789
:101AA6009BEC9AE899400AED9BFDEC9AFCE899F8C4
:0E1AB6000FD5F0DAE4CDFBE4CCFAE4C8F92257
:10A64D00C2D5E830E70FB2D5E4C39BFBE49AFAE438
:10A65D0099F9E498F8EC30E717B2D512A683121ADF
:10A66D0032E4C39BFBE49AFAE499F9E498F8800389
:10A67D00121A3230D50DE4C39FFFE49EFEE49DFD1A
:04A68D00E49CFC222B
:0D1AC400CFF4CFCEF4CECDF4CDCCF4CC22B7
:101AD100E8600FECC313FCED13FDEE13FEEF13FFF3
:031AE100D8F12217
:101AE400E86010ECA2E713FCED13FDEE13FEEF1318
:041AF400FFD8F02205
:101AF800E8600FEFC333FFEE33FEED33FDEC33FC4C
:031B0800D8F122EF
:101B0B00BB010789828A830220B95005E9F8021BC1
:101B1B0099BBFE05E9F80220C589828A830220D190
:101B2B00BB010DE58229F582E5833AF5830220B9E5
:101B3B005007E92582F8021B99BBFE07E92582F8BD
:101B4B000220C5E58229F582E5833AF5830220D18F
:101B5B00BB010789828A83021BEE5005E9F8021B41
:0A1B6B00E2BBFE05E9F802210A22A0
:101B7500BB010DE58229F582E5833AF583021BEE6B
:101B85005007E92582F8021BE2BBFE07E92582F82A
:041B950002210A22FD
:0C1B9900E6FC08E6FD08E6FE08E6FF2278
:0D1BA500E6FB08E6F908E6FA08E6CBF822B0
:101BB200BB010DE58229F582E5833AF5830220E136
:101BC2005007E92582F8021BA5BBFE07E92582F82A
:101BD2000220EDE58229F582E5833AF5830220FAB7
:0C1BE200ECF608EDF608EEF608EFF6222F
:0C1BEE00ECF0A3EDF0A3EEF0A3EFF0226A
:101BFA00A8828583F0D083D082121C11121C111284
:101C0A001C11121C11E473E493A3C583C5F0C583A8
:101C1A00C8C582C8F0A3C583C5F0C583C8C582C834
:011C2A002297
:101C2B00BB010DE58229F582E5833AF58302212874
:101C3B005007E92582F8022116BBFE07E92582F839
:101C4B00022168E58229F582E5833AF58302217A40
:101C5B00BB0120E58229F582E5833AF583D0F0D0EC
:101C6B00E0F8D0E0F9D0E0FAD0E0FBE8C0E0C0F05B
:101C7B0002215F5018E92582F8D083D082D0E0F999
:101C8B00D0E0FAD0E0FBC082C08302211FBBFE185C
:101C9B00E92582F8D083D082D0E0F9D0E0FAD0E009
:091CAB00FBC082C08302217122FA
:101CB400D083D082F8E4937012740193700DA3A3BF
:101CC40093F8740193F5828883E4737402936860D3
:061CD400EFA3A3A380DFD3
:061CDA008A838982E47395
:101CE000E5132582F582E5123583F583B512048567
:101CF00082132210AF06858213F51222858213F516
:041D000012D2AF222A
:0D1D0400E5132582F582E5123583F5832273
:10A4E00090FE6D1220B97810EC4D4E4F70047CA593
:10A4F0007DA5C3EC13FCED13FDEE13FEEF13FF502F
:10A5000010EC64CCFCED644CFDEE644EFEEF64CECA
:10A51000FFD8DF90FE6D121BEEEE547FFE2290FE00
:0DA520006DEEF0EFA3F0A374A5F0A3F02200
:1063EE00E508302C0104F8232824F8F582E434FB68
:1063FE00F5832290FBF5302C0390FBF8E475F00149
:10640E0012213102176660EAC50C7002150B14C515
:10641E000C202C04FF02B39B90FBF574FFF5F002E9
:10642E002148FF02B246E5096006D509037F002226
:10643E00202C0F12B232EF6008050CE50C7002052D
:10644E000B2290FBF5122128121766FF60E890FBD5
:10645E00F5E475F00112213180DC12643EEFC0E0EC
:10646E00126430D0E040F3809DD22C8002C22C907A
:10647E00FBF512215FE4F50AF508F50BF50C75092D
:10648E0000C22BC229C22AC22D126401FF7005AFB1
:10649E000A7E0022B42530126401FF24D0B40A0013
:1064AE00500C75F00AC509A42509F50980E924CF19
:1064BE00B41A00EF5002C2E50266DCD22A80D8D2AE
:1064CE002980D4D22D80D0EF126430500812646827
:1064DE00EF600E80A9EFC0E012643ED0E06F609EC8
:1064EE00EF607412641480A712643EEF6069E509D0
:1064FE0070070509800312643EEF6014202D0E1202
:10650E0063EEE475F001122131EF1217ACD509E6F6
:10651E00202D040508050A80BA126434EFC0E0127B
:10652E006430D0E05004126414E4FF202D0E126388
:10653E00EEE475F001122131EF1217ACEF70DA2094
:10654E002D040508050A808BE50960020509126411
:10655E0068126434EF70C6302C04E4126414E50A39
:10656E00600302649D7EFF7FFF22202D1174FFFCCD
:10657E00FDFEFF1263EE122128121B5B050802645A
:10658E008CD0E080D27900800A791080067908805C
:10659E0002790AD22EE50960020509E9C0E012640B
:1065AE0068EF60DD12643EBF2D04D22B8003BF2B3B
:1065BE0009126468EF60CA126434D0E0B40A028033
:1065CE0033B40802802EBF302770027408C22EC06A
:1065DE00E0126434D0E0BF78028003BF581605097C
:1065EE00D509028007D50904D22E800B74108019AC
:1065FE007002740ABF000AEFF8E4FCFDFEFF0266AB
:10660E008FC0E0EF126414D0E0F9E4FCFDFEFFE968
:10661E00C0E0ECC0E0EDC0E0EEC0E0EFC0E0126420
:10662E0034EFF8D0E0FFD0E0FED0E0FDD0E0FCD0BB
:10663E00F0E8604DB461004007B47B005002C2E543
:10664E0024D0503DFA24F6500724F95034240AFA87
:10665E00EAB5F000502BCFA9F0A42FFF92D5E9C5D3
:10666E00F0CEA4A2D53EFE92D5E9C5F0CDA4A2D51A
:10667E003DFD92D5E9C5F0CCA4A2D53CFCC22E803E
:06668E008EE8C0E0202DA3
:106694002A202E08050A302B031220AB1263EE12B7
:1066A4002128050820290B202A0DEE8FF012208CBA
:1066B4008009121B5B8004EF1217ACD0E012641443
:1066C40002648C202D101263EE1221280508E50BBC
:1066D400850CF012208C80E8121CB4655653659723
:1066E4005864CD4C64C94264A548659B4F659F447A
:1066F40064F643659349659F5565784665784565B5
:0C670400784764D12A66C74E000064D5B7
:101D1100E3F5F009E208B5F06D606B80F3E3F5F0EF
:101D210009E608B5F060605E80F387F009E608B562
:101D3100F054605280F487F009E208B5F04860463B
:101D410080F488828C8387F009E0A3B5F03860368F
:101D510080F488828C8387F009E493A3B5F027602F
:101D61002580F388828C83E3F5F009E0A3B5F016B2
:101D7100601480F388828C83E3F5F009E493A3B5C2
:101D8100F004600280F2021E3C808580E7808E8034
:101D9100D2803C8015806C807E809B80B5808B805A
:101DA100A1804F8070803A021E5289828A83ECFAA8
:101DB100E493F5F0A3C8C582C8CCC583CCE493A352
:101DC100C8C582C8CCC583CCB5F070606E80E1898E
:101DD100828A83E493F5F0A3E208B5F05E605C804B
:101DE100F289828A83E0F5F0A3E608B5F04D604BF5
:101DF10080F389828A83E0F5F0A3E208B5F03C60C4
:101E01003A80F389828A83E493F5F0A3E608B5F07A
:101E11002A602880F2805D89828A83ECFAE493F556
:101E2100F0A3C8C582C8CCC583CCE0A3C8C582C80D
:101E3100CCC583CCB5F004600280E27F00F845F0A8
:101E4100600EE863F0806480D395F01F40027F014B
:101E51002289828A83ECFAE0F5F0A3C8C582C8CC56
:101E6100C583CCE0A3C8C582C8CCC583CCB5F0CBB3
:101E710060C980E389828A83ECFAE0F5F0A3C8C5E2
:101E810082C8CCC583CCE493A3C8C582C8CCC58322
:101E9100CCB5F0A760A580E288F0ED2402B404007F
:101EA1005099F582EB2402B40400508F232345821C
:051EB10023901D8A735F
:10B20900E4FFFE121766600C0FEF70010E09E9707A
:05B21900F20A80EF22A3
:101EB600E3F5F009E208B5F06BDFF58067E3F5F0CE
:101EC60009E608B5F05EDFF5805A87F009E608B541
:101ED600F052DFF6804E87F009E208B5F046DFF6ED
:101EE600804288828C8387F009E0A3B5F036DFF65E
:101EF600803288828C8387F009E493A3B5F025DFCE
:101F0600F5802188828C83E3F5F009E0A3B5F0140F
:101F1600DFF5801088828C83E3F5F009E493A3B59E
:101F2600F002DFF4021FE5808780E9809080D4808C
:101F36003E8015806E807E809D80B7808D80A380D8
:101F4600518074803C021FF189828A83ECFAE49303
:101F5600F5F0A3C8C582C8CCC583CCE493A3C8C595
:101F660082C8CCC583CCB5F076DFE3DEE18070892C
:101F7600828A83E493F5F0A3E208B5F062DFF48089
:101F86005E89828A83E0F5F0A3E608B5F051DFF5B5
:101F9600804D89828A83E0F5F0A3E208B5F040DF40
:101FA600F5803C89828A83E493F5F0A3E608B5F0D0
:101FB6002EDFF4802A8002805789828A83ECFAE435
:101FC60093F5F0A3C8C582C8CCC583CCE0A3C8C529
:101FD60082C8CCC583CCB5F006DFE4DEE280007FA4
:101FE600FFB5F0020F2240027F012289828A83EC2C
:101FF600FAE0F5F0A3C8C582C8CCC583CCE0A3C877
:10200600C582C8CCC583CCB5F0D5DFE5DEE380CF8D
:1020160089828A83ECFAE0F5F0A3C8C582C8CCC5EC
:1020260083CCE493A3C8C582C8CCC583CCB5F0AF36
:10203600DFE4DEE280A988F0EF60010E4E60ABEDD2
:102046002402B404005098F582EB2402B404005034
:0A2056008E2323458223901F2D7373
:10206000EF4E6012EF60010EEDBB010B89828A8397
:10207000F0A3DFFCDEFA2289F05007F709DFFCA9A4
:0C208000F022BBFEFCF309DFFCA9F022FB
:10A5780090FE1AE0FFA3E0FEA3E0CF90FC51F0A309
:10A58800EEF0A3EFF090FE1DE0CBF0A3E0CAF0A33D
:10A59800E0C9F07F2290FC54AD82AC831217668D1F
:10A5A800828C83F0A309E970010ADFEC90FE1DE0BC
:0AA5B800FBA3E0FAA3E0F90260EE55
:109769000234EBE493A3F8E493A34003F68001F2F7
:1097790008DFF48029E493A3F85407240CC8C33301
:10978900C4540F4420C8834004F456800146F6DFD0
:10979900E4800B01020408102040809087CCE47E0D
:1097A900019360BCA3FF543F30E509541FFEE493C5
:1097B900A360010ECF54C025E060A840B8E493A38C
:1097C900FAE493A3F8E493A3C8C582C8CAC583CAB7
:1097D900F0A3C8C582C8CAC583CADFE9DEE780BE6F
:0188980000DF
:10208C00BB010A89828A83F0E5F0A3F0225006F79F
:0F209C0009A7F01922BBFE06F3E5F009F319229C
:0E20AB00C3E49FFFE49EFEE49DFDE49CFC2246
:0C20B900E0FCA3E0FDA3E0FEA3E0FF229A
:0C20C500E2FC08E2FD08E2FE08E2FF2257
:1020D100E493FC740193FD740293FE740393FF2255
:0C20E100E0F8A3E0F9A3E0FAA3E0FB2282
:0D20ED00E2FB08E2F908E2FA08E2CBF82273
:1020FA00E493F8740193F9740293FA740393FB223C
:0C210A00ECF208EDF208EEF208EFF22211
:09211600E6FB08E6FA08E6F922EE
:09211F00EBF608EAF608E9F622E5
:09212800E0FBA3E0FAA3E0F922B8
:10213100F8E0FBA3A3E0F925F0F0E5821582700237
:072141001583E0FA38F022DB
:10214800F8E0FBA3A3E025F0F9F0E5821582700220
:072158001583E038FAF022C4
:09215F00EBF0A3EAF0A3E9F02281
:09216800E2FB08E2FA08E2F922A8
:09217100EBF208EAF208E9F2229F
:0C217A00E493FB740193FA740293F922C1
:10608900E50D2451F582E434FCF583E0050D2290F9
:10609900FC4E30270390FC51E475F00112213102C6
:1060A90017662020E97F2ED2208018EF540F249004
:1060B900D43440D4FF30240BEF24BFB41A0050036A
:1060C9002461FFE50E6002150E0511E51170020548
:1060D9001030270E90FC4EE475F001122131EF02C9
:1060E90017AC02AE767403D2278003E4C227F50DFC
:1060F90090FC4E12215FE4F50EF510F511E50E60E6
:10610900077F201260CC80F5750FFFC221C220C223
:1061190022C223C225C226C228126098FF700D3000
:1061290027057F001260DDAF11AE1022B4255FC2D2
:10613900D5C224126098FF24D0B40A00501A75F011
:106149000A780E30D50508B6FF0106C6A426F62042
:10615900D5047002D22380D924CFB41A00EF500499
:10616900C2E5D2240262DED22180C6D22080C0D20A
:106179002280BCD2D580BAD22580B47F201260CCCF
:106189002022077401B50E0040F1126089FF1260E8
:10619900CC026106D228D2268095126089FB126052
:1061A90089FA126089F94A4B700679AF7A637BFFE5
:1061B90020222EE50E602A7E008E8275830012173A
:1061C9007F60060EEE650F70F0C2D5EBC0E0EAC045
:1061D900E0E9C0E0EE126325D0E0F9D0E0FAD0E0C2
:1061E900FB121766FF60AAEBC0E0EAC0E0E9C0E075
:1061F9001260CCD0E02401F9D0E03400FAD0E0FB01
:10620900E50F0460DCD50FD980877BFF7A6379219C
:10621900D222809C791080027908C226C22880087F
:10622900D2D5790A8004790AC2D5E50F047002F53E
:106239000FE4FAFDFEFF126089FC7B08202113128E
:106249006089FD7B1030200A126089FE126089FF87
:106259007B20EC3382D592D55013C3E43020069FBE
:10626900FFE49EFEE42021039DFDE49CFCE4CBF8C1
:10627900C221EC700CCFCECDCCE824F8F870F380B5
:1062890017C3EF33FFEE33FEED33FDEC33FCEB3395
:10629900FB994002FB0FD8E9EB302105F8D0E0C4A7
:1062A90048B221C0E00AEC4D4E4F78207B0070C205
:1062B900EAB50F0040BCC0E0126327D0F0D0E0205F
:1062C9002104C4C0E0C4B221C0F01260B5D0F0D539
:1062D900F0EB026106121CB461A353621D5861748C
:1062E9004C61704262214F622944622949618943A4
:0862F900622F55621346621387
:106301004562134763CF5061782D617C2E619F2BCD
:10631100618023619D2063B82A613848000061973C
:106321003F3F3F00790AA2D5202314302509B91037
:10633100020404B9080104A2D52026025001042058
:1063410022689222B50E005034C0E07F203023191C
:106351007F30A22272267225500F12637EC222C2A2
:1063610026C225C2287F30800F302503E9C0E01204
:1063710060CC302503D0E0F9D0E0B50ECC30251744
:106381007F30B9100C1260CC7F583024077F7880A1
:1063910003B908031260CC3022057F2D0260CC7F47
:1063A100202028F87F2B2026F322922280CF286EEE
:1063B100756C6C2900D2211260893021F8C22178D4
:1063C1000E30D50108F60261382D5043495812604C
:1063D100892403B405004001E49063CA931260BDAF
:0D63E100743A1260BDD223750E0402621DD5
:10B2320010330B12B381BF0D027F0A02AE7690FE6D
:04B24200FCE0FF220B
:08B39B0090FEFCEFF0D233221A
:10B24600EFC394094005EF940E4004EFB42003D3F6
:04B256008001C3228E
:10AE7600EFB40A07740D12AE81740A309811A899BE
:10AE8600B8130CC2983098FDA899C298B811F6303C
:07AE960099FDC299F5992214
:0AB381003098FDAF99C2987E0022BB
:00000001FF
